:020000040800F2
:10000000E01C0020B5780008F5780008D31500083A
:10001000F9780008FB780008FD780008000000006F
:10002000000000000000000000000000FF78000851
:10003000017900080000000003790008555C000801
:100040000779000807790008077900080779000890
:10005000077900080779000807790008C3640008D9
:100060000779000807790008077900080779000870
:1000700007790008077900086F5E00080779000813
:100080000779000807790008077900080779000850
:10009000077900080779000807790008C564000897
:1000A00007790008077900080779000879580008DF
:1000B000655900086D590008735900084354000839
:1000C00021520008475400084554000807790008E9
:1000D00007790008077900089B6000080779000885
:1000E000554D00080779000807790008DFF80CD0A3
:1000F00008F024F90048004781140008E01C0020A3
:1001000070B51546B0FBF5F60446A84203D3304659
:10011000FFF7F6FF014605FB1640F8A2105C0870D9
:10012000481C70BD70B50C46911E232900D30A22CD
:100130000025002804DA2D212170611C404200E0D6
:100140002146FFF7DDFF0570204670BD70B50546FE
:100150000C46086807F05DFC024621682868BDE887
:10016000704007F05EBC10B5EEA005F04DFF012019
:1001700000F0A3FDF2A005F047FF0A2005F092FD74
:10018000BDE81040002005F033BE10B5F0A005F02A
:100190003BFF002000F065FDF0A005F035FF0A20D0
:1001A00005F080FDBDE81040002005F021BE10B52F
:1001B0000446EEA005F028FF2021F24807F0FEFBE0
:1001C000F14800210160F14801702046BDE810406F
:1001D000DBE72DE9F047064607F01BFC054600F07B
:1001E0007DFEDFF8A49307464FF0010809F150099E
:1001F00055B12A46E6A1304607F013FCD8B1307855
:1002000000272D2827D029E0E3A005F0FDFE0024DB
:1002100045464E4656F8241059B105FA04F03842C6
:1002200002D0084605F0F0FE202005F0E0FE641C38
:10023000F0E7C2A01FE0DDA005F0E6FE00244D4679
:1002400055F824000028F4D005F0DEFE202005F04B
:10025000CEFE641CF4E70127761C6D1E5FF00004DF
:1002600059F8241031B12A46304607F0DAFB30B194
:10027000641CF5E7D3A0BDE8F04705F0C5BE08FA59
:1002800004F01FB100F025FED5A002E000F010FD43
:10029000D6A005F0B9FE59F8240005F0B5FEC8E770
:1002A00070B50024D4A005F0AFFED94D04EB440690
:1002B00055F8260005F0A8FE092005F098FE05EB8C
:1002C0008600406805F0A0FE9CA005F09DFE00BFE2
:1002D00005F077FE0028FBD0641C0A2CE6D370BD25
:1002E0003EB5054607F095FB08281BD10024285D84
:1002F00007F022FB2855641C082CF8D30024C548BD
:10030000295D07F07DFB28B12819295D401C07F005
:1003100077FB08B1C0A01AE0641C082CEFD3284674
:1003200000F01AFCC4A005F06FFEBA4BC84A0020CA
:10033000694615181C5C95F86D50401C08284C55F2
:10034000F7D300220A54084605F05EFE7BA005F0B4
:100350005BFE3EBD2DE9F041804607F05AFB8A4D19
:10036000BB4F10F0FF0605F1040512D0324688A1FC
:10037000404607F056FBA8B15FF0000455F8241082
:1003800009B33246404607F04CFB08B3641CE4B2A4
:10039000F4E7B0A005F038FE787805EB800050F85F
:1003A000040C1CE0AFA005F02FFE002455F824003B
:1003B00038B105F029FE202005F019FE641CE4B2D6
:1003C000F4E75EA000E0ACA0BDE8F04105F01CBE83
:1003D000601C7870AEA005F017FE55F8240005F0FB
:1003E00013FEEEE77FB504460D462179002005296E
:1003F00014D2DFE801F003060A0D1100A0680078AE
:100400000CE0A06890F9000008E0A068008805E012
:10041000A068B0F9000001E0A06800680A226946FF
:10042000FFF780FE684605F0EFFD002D15D06EA0A9
:1004300005F0EAFD0A226946E068FFF773FE6846A8
:1004400005F0E2FD68A005F0DFFD0A22694620699B
:10045000FFF768FE684605F0D7FD7FBD2DE9F04740
:10046000814607F0D6FA6A4C060004F1780425D0DC
:10047000012E03D199F800002A281FD088A14846F0
:1004800007F0A8FA002836D0401C07F0E3FA8046AF
:100490005FF0000505EB850704EB870654F827009D
:1004A00007F0B7FA024654F82710484607F0B9FAA1
:1004B00018B36D1C462DEDD37AA03BE181A005F069
:1004C000A3FD002505EB850004EB800754F8200010
:1004D00005F09AFD81A005F097FD31463846FFF7FB
:1004E00081FF16A005F090FD05F06BFD0028FBD004
:1004F0006D1C462DE6D3BDE8F087F1E03031323394
:100500003435363738394142434445464748494AED
:100510004B4C4D4E4F505152535455565758595AB3
:1005200000000000526573657474696E6720746F13
:100530002064656661756C74732E2E2E0D0A0000A2
:100540005265626F6F74696E672E2E2E0000000078
:10055000536176696E672E2E2E0000000D0A5265DB
:10056000626F6F74696E672E2E2E00000D0A4C6547
:100570006176696E6720434C49206D6F64652E2E4D
:100580002E0D0A0078040020000000204102002007
:100590006C69737400000000456E61626C656420D4
:1005A00066656174757265733A2000004176616911
:1005B0006C61626C652066656174757265733A2062
:1005C00000000000496E76616C69642066656174A4
:1005D000757265206E616D652E2E2E0D0A0000006D
:1005E00044697361626C656420000000456E61625D
:1005F0006C65642000000000417661696C61626C8A
:100600006520636F6D6D616E64733A0D0A000000C2
:1006100080970008709D00084D75737420626520F6
:10062000616E79206F72646572206F662041455457
:1006300052313233340D0A0043757272656E742084
:1006400061737369676E6D656E743A200000000017
:100650009804002043757272656E74206D69786528
:10066000723A2000417661696C61626C65206D6947
:10067000786572733A200000496E76616C69642077
:100680006D6978657220747970652E2E2E0D0A00C2
:100690004D697865722073657420746F20000000C6
:1006A0003D0000004552523A20556E6B6E6F776EDA
:1006B000207661726961626C65206E616D650D0AFC
:1006C0000000000043757272656E74207365747467
:1006D000696E67733A200D0A00000000203D20007B
:1006E00005EB850104EB8100C368434521DC026909
:1006F00042451EDB3279052A0FD2DFE802F0030300
:1007000007070B00B26882F8008006E0B268A2F822
:10071000008002E0B268C2F8008054F8210005F0C1
:1007200073FCADA005F070FC3046BDE8F047002139
:1007300058E6ACA0BDE8F04705F066BC2DE9FF41E6
:10074000B2A005F061FC05F09FFA4FF47A71B0FB9E
:10075000F1F00A226946FFF7E5FC684605F054FC13
:10076000AEA005F051FCB2480A2269460078FFF7B6
:10077000D9FC684605F048FCAEA005F045FCB04841
:100780000A2269460078FFF7CDFC684605F03CFC7C
:10079000ACA005F039FC00F091FB0646ADA005F0D9
:1007A00033FC0024B04F012557F8240058B105FA56
:1007B00004F1314201D005F027FC202005F017FCA0
:1007C000641CE4B2F0E7012000F066FB50B1A7A082
:1007D00005F01AFCA749A4480978183050F8210000
:1007E00005F012FCAFF2AC2005F00EFCA2A005F063
:1007F0000BFCA5480A2269460088FFF793FC68466F
:1008000005F002FCA1A005F0FFFB04F0A5FE0A2202
:100810006946FFF787FC684605F0F6FBAFF2E42077
:1008200005F0F2FBBDE8FF819CA005F0EDBB2DE9D2
:10083000FF5FDFF8989299F8000038B9012189F834
:100840000010A3A005F0E0FB00F0C3F8DFF818A249
:10085000DFF8B4B2AAF1840A05F0A6FB00286ED036
:1008600005F0B8FB092806D03F2804D0DAF80010BC
:100870005446B1B34DE0A54F0024254607F1780852
:10088000DAF800600CE000BFDAF8002022B19E48E0
:10089000396807F0C6F810B904B93C463D460C3734
:1008A0004745F1D39CB150465F46016822682B68EA
:1008B000525C5B5C9A420AD11AB17A54491C0160BD
:1008C000F3E720220BF80120491CCAF80010DAF8DF
:1008D0000000574608B1AC4210D08DA005F094FB43
:1008E00007E014E0206805F08FFB092005F07FFB8E
:1008F0000C34AC42F6D900F06CF800265C4638683F
:100900008642A9D2A05D05F072FB761CF7E70428A9
:1009100010D00C2814D019B10A2815D00D2813D0E6
:100920007F283ED0202997D2202895D37E2893D89F
:10093000B1B344E004B07448BDE8F05F37E446E08A
:1009400075A005F061FB28E0AFF2104005F05CFBFC
:10095000206800255E460BF800507248CDE9000B78
:100960000C230A226949029501A806F0EBFF070053
:1009700007D0386807F04DF83044B968401C884704
:1009800002E069A005F040FB20215F4807F016F85F
:10099000256099F80000002819D000F01AF85BE7EC
:1009A0000BE00029FBD0491E0020CAF800100BF80C
:1009B000010066A005F028FB4EE72028EFD00BF8D9
:1009C0000100491CCAF8001005F011FB44E7BDE81E
:1009D000FF9F5FA005F018BB2073657420746F2023
:1009E000000000004552523A2056616C7565206146
:1009F000737369676E6D656E74206F7574206F66B2
:100A00002072616E67650D0A0000000053797374EF
:100A1000656D20557074696D653A200020736563BB
:100A20006F6E64732C20566F6C746167653A20009A
:100A30003C010020202A20302E31562028000000C2
:100A4000E8010020532062617474657279290D0AEF
:100A50000000000044657465637465642073656E0E
:100A6000736F72733A2000008400002041434348B2
:100A7000573A2000F40100204379636C65205469E3
:100A80006D653A20000000003E0100202C20493214
:100A900043204572726F72733A2000004166726F94
:100AA000333220434C492076657273696F6E203271
:100AB0002E30204175672032312032303132202FE4
:100AC0002031323A35393A313900000041020020F4
:100AD0000D0A456E746572696E6720434C49204D5E
:100AE0006F64652C20747970652027657869742798
:100AF00020746F2072657475726E2C206F722027BF
:100B000068656C70270D0A00780400208097000843
:100B10000D1B5B4B000000001B5B324A1B5B313B33
:100B2000314800004D0100084552523A20556E6B85
:100B30006E6F776E20636F6D6D616E642C207472C2
:100B400079202768656C70270000000008200800E5
:100B50000D0A2320000000002DE9F041054604465F
:100B6000E04EE14F09E0DF4806F04AFF20B1611B8B
:100B7000801B384480F86D10641C21780029F2D164
:100B8000BDE8F0812DE9F05FD422D849D64806F0BF
:100B9000FCFED548D64E002190F8292090F8284038
:100BA00040F6C41501FB01F3193B534303F6C4138C
:100BB0004B43634393FBF5F326F81130491CC9B24C
:100BC0000629EFD390F82B20B0F886409246C2F168
:100BD000640C90F82A30B0F888200021DFF814B3B4
:100BE0004FF00A0E03EB8308A146151B01EB8102AF
:100BF000C3EB42040122002C03DDC3F16402D2B234
:100C000001E000DA1A4604FB04F70AFB07F602FBD0
:100C100002F296FBF2F2624402FB04F292FBFEF255
:100C200002EB480212B205FB02F24FF47A7492FB17
:100C3000F4F404EB09022BF8112001F10101C9B20F
:100C40000B29D3D3B0F8AA10B0F8AC20914203D34B
:100C5000B0F8AE20914200D91146A0F8AA10BDE824
:100C6000F09F2DE9F041064606F0B0FD342006F075
:100C700017FE9E4D284606F0D7FD04280AD19A4F4C
:100C800000246019395906F0EBFD042802D1241D17
:100C9000D42CF6D306F0A0FDFFF774FF002E06D08B
:100CA000BDE8F041012214210F2001F089B867E767
:100CB0008D494A6802434A6070472DE9F05F8B49CD
:100CC0000A788D49097808B98A427CD0864C03207D
:100CD00000252170607002206560FFF7E9FF258123
:100CE0002821A1724FF01E0B84F814B0083417228B
:100CF000A275E17084F80DB0E275552020712D22A7
:100D0000A2732576102060710F20E07307206076B3
:100D10000B20A0712574A5761427E771082363744E
:100D2000E2760E222272A774502222774622627245
:100D30004FF00A0A84F813A06777A172E57265750F
:100D4000E5775A2084F82000412084F8210084F8B7
:100D5000245084F8255084F826504FF0320984F846
:100D6000229084F82350A4F108044FF0000000BF43
:100D700004EB400100F10100C0B2A1F84E500E2872
:100D8000F6D304F164044FF0040024F8265C24F840
:100D9000245C24F8345C24F8325C24F8305C24F8B9
:100DA000285C04F8225C04F8210C4FF4C87824F87D
:100DB0001E8C4FF02A0024F8200C4FF0010604F896
:100DC000186C4E4800E066E044F81C0C4FF06E00D2
:100DD000A0714FF02B00E0714FF02100207248A06D
:100DE000FFF7BAFE6574A574E774257540F2DC5010
:100DF000E08240F24C41218340F26C71618325779F
:100E00003A4684F81DA0C827A7774FF49663238439
:100E100040F27E43638440F23A73A3844FF47A73C2
:100E2000E384A4F82880A4F82A9084F84460A4F805
:100E300046004FF47F73A4F848304FF4FA655146EA
:100E4000A4F84A5084F84C1084F84D1084F84E6091
:100E5000A4F85030A4F85250A4F85400A4F8563026
:100E6000A4F85850A4F85A004FF41650E065A4F8BE
:100E7000607084F8622084F863B004F8646F6420C2
:100E800060804FF49670A0804FF4E130A060BDE820
:100E9000F05F0020E5E6E2E617494968014201D02B
:100EA000012070470020704713494A6802434A6096
:100EB000704711494A6882434A6070470E4840684B
:100EC000704709494968014201D00120704700205C
:100ED000704705494A6882434A6070470248406843
:100EE00070470000709D00089804002000FC010875
:100EF0005807002064070020B000002003141400ED
:100F0000414554523132333400000000FD4810B5E1
:100F1000008806F099FFFC4906F001FE06F099FFF3
:100F2000FA4908800420FFF7B7FF002803D0BDE886
:100F3000104002F0A3B810BD2DE9F04706460C465C
:100F4000D6E9007080464868B568414606F0E7FD7E
:100F500081463946206806F0E2FD494606F087FDE5
:100F6000294606F0D9FDB0604146A06806F0D7FDDD
:100F700081462946206806F0D2FD494606F0C9FDA3
:100F8000394606F074FD30603946A06806F0C7FDAA
:100F900007462946606806F0C2FD394606F067FD3F
:100FA000414606F064FD7060BDE8F0872DE9F04F22
:100FB00089B0002504F053FED44F06463C46B8697C
:100FC000301A06F041FFD24906F0A9FD0290A66151
:100FD000DFF8408300240DF1180B07F1500A4FF0A1
:100FE0007E5907F15606C9484A3030F9140006F018
:100FF00022FF029906F093FD4BF8240098F8430075
:1010000000B306F021FF0146484606F0BEFD0490FD
:101010003AF9140006F00FFF049906F080FD0390E2
:101020004946049806F078FDBB4951F8241006F0B3
:1010300076FD039906F01BFDB74941F8240006F040
:1010400008FF01E03AF8140026F8140036F91400FD
:1010500000FB00550420FFF71FFF641C032CC2D3C4
:1010600064204543A74806A90088404395FBF0F457
:10107000A9481838FFF760FF0420FFF70DFF20B1E3
:10108000A54806A90C38FFF757FFB6F9000000285D
:1010900000DC4042B7F90020A049BA4690420CDA81
:1010A000B6F90200002800DC4042904205DAB6F9A9
:1010B0000400002801DD012000E00020964D253CC1
:1010C000183D48739F2C02D310F0FF0F23D000244B
:1010D0004F46B8F8460006F0B7FE8146394606F09E
:1010E000C6FC0146384606F050FD804636F914002D
:1010F00006F0A1FE074655F82410484606F00FFDFD
:10110000394606F0B4FC414606F009FD45F82400D6
:10111000641C032CEAD30420FFF7BEFE7E4E0C3E77
:10112000E8B1DFF8E881DFF8F891DFF8F8B10024E2
:1011300008F15C0838F9140006F07DFE074656F801
:101140002400494606F0EBFC394606F090FC59466F
:1011500006F0E5FC46F82400641C032CEAD3A968D9
:10116000286800F077F9694C10342080D5E9010136
:1011700000F070F960800420FFF78EFE002837D061
:10118000B4686868214606F0CAFCAF68804671689A
:10119000384606F0C4FC414606F0BBFC80463846A3
:1011A000316806F0BCFC06462146286806F0B7FC0C
:1011B000314606F0AEFC414600F04CF95A4C06F0C0
:1011C0003AFEDAF80C1006F052FC06F042FE00B2CD
:1011D0000A2190FBF1F000B22080B42802DDA0F5D6
:1011E000B47004E010F1B40F02DA00F5B47020809E
:1011F00009B0BDE8F08F2DE9FF5F0120FFF74CFE3D
:1012000018B101F04EFEFFF7D1FE01F01AFF0025E4
:101210003E4C6F464A34AA4604F1060B34F81500DA
:1012200027F815000120FFF737FE08B92BF815A0A5
:101230006D1C032DF2D304F012FD344E706100F0EA
:10124000E9FD04F00CFD716940F28A25401AA842BC
:1012500004D936480188491C018005E004F0FFFCF0
:101260007169401AA842F9D301F0EBFEA046B946D5
:10127000264C00250327383438F8151039F81500A6
:10128000084402A900B221F8150020493E3131F985
:101290001520024492FBF7F200EBD07024F81520E1
:1012A000401021F815000120FFF7F6FD08B92BF8D2
:1012B00015A06D1C032DDFD34020FFF702FE154A59
:1012C000B0B312490831087828B9906C020C0A7042
:1012D000020A4A7088700D4D002044350A5C34F9CA
:1012E000106035F91070531E07FB03635B1C93FB02
:1012F000F2F224F8102025F81020401C0328EDD32A
:10130000BDE8FF9FFC0100207593D83EB800002087
:10131000534492319804002084050020480700209F
:10132000000048435E06A33B3C020020E40100208D
:10133000FFE750780128E3D1B4F90400B6F90610AC
:1013400000EB410090FBF7F0A080F080D8E7F0B50B
:10135000454801684548C2698A1A7AD446F2A812FB
:101360001144C161C26A0A2492FBF4F2404B016A43
:1013700012B233F9115023F81120446A161901F101
:1013800014022824B2FBF4F704FB1722491C33F99A
:101390001220B31A4362866A3244551B00268562C6
:1013A0000162282900D3066232495D1B91F8212091
:1013B0006A4392FBF4F2524214B203EB83025200EE
:1013C000142392FBF3F244800263436B9A1A002ABF
:1013D00001DD134600E053420A2B03DA0934122CD4
:1013E00000D846804B7B5C42B2EB440F02DA5C00D3
:1013F000644205E0B2EB430F01DD5C0000E01446FF
:101400006343642493FBF4F3448823441BB26FF0DA
:1014100095044380A34201DA234602E0962B00DDC7
:1014200096234380C97D5143322291FBF2F1828899
:10143000114409B2104A8180914202DB524291422A
:1014400000DD114681804FF4FA7291FBF2F11944EC
:101450004180F0BD10B507F0B1F9084906F05FFB17
:1014600006F0F7FC00B210BD5C010020B8000020BF
:101470009005002098040020D08AFFFF4C3D0F44C7
:101480000EB504F01AFCFFF77DFB0020FFF715FCFA
:10149000534CD4F8D00001F0D8FF0720FFF704FD2B
:1014A00000F0B4F860784FF001080E2801D0082849
:1014B00001D18DF804800120FFF703FD8DF80100B4
:1014C0000820FFF7FEFC80F001008DF80000454881
:1014D000007800B101208DF8020094F8B200C0F34A
:1014E000C0008DF80300B4F88C00ADF80600B4F825
:1014F0008E00ADF80800684604F087FADFF8EC903B
:1015000039494FF0100AC9F800103949C1F800A054
:101510000E1F4FF0080BC6F800B000258F1434489A
:101520000838016881F010010160016881F008014C
:101530000160192004F0B6FB2E480760192004F062
:10154000B1FB2C48001F07606D1CEDB20A2DE6D3DD
:10155000C6F800B0C6F800A001F006FBFFF7D6FC05
:101560000220FFF7AEFC08B101F0B7FB0820FFF73F
:10157000A8FC28B103F057F81F49C9F8001013E080
:101580000120FFF79EFC78B14FF48070FFF799FCC3
:1015900018B1D4F8C00002F04CFF4FF48060FFF7A0
:1015A00090FC08B101F097FE04F059FB1349086064
:1015B0006078052803D112494FF4C870088011499A
:1015C0004FF47A700880104981F80D8000F04CFECD
:1015D000FCE70348B0F98A0000F095F8FEE7000048
:1015E00098040020230100208321000864010020CA
:1015F000140C0140140801404F460008600100200F
:10160000F8010020FA0100204807002070B5FC4EC8
:101610000125FC4C7078042807D0012805D0082843
:1016200003D00E2801D0052800D165702020FFF7D7
:1016300048FC00B165707178002013290CD2DFE8F6
:1016400001F00B0E10100C1512120A1012141414C3
:101650000A0B0B101700257070BD022006E0032056
:1016600004E0042002E0062000E00820207070BDA5
:101670002070E54A002000BF00EB800112F8211025
:1016800011B12178491C2170401C0C28F4DB70BD7D
:10169000DC4810B54078002823D0D948D94C407890
:1016A000A41C01281AD0042812D0082819D00E280A
:1016B00017D02020FFF705FC002812D02188002039
:1016C00004F01BFA61880120BDE8104004F015BA4F
:1016D0002189002004F011FA6189F4E76189002072
:1016E000F2E710BD70B5C84E0024183EC54D06E0A7
:1016F00036F81410204604F0F4F9641CE4B228789B
:101700008442F5D370BDBF4ABF4B00211278183B0D
:1017100004E000BF23F81100491CC9B29142F9D37B
:10172000E0E72DE9F04FB748B84F97B000780328AD
:1017300023D9B748B7F90420B0F904004142002882
:1017400001DD034600E00B466FF06304E31A9A42A2
:1017500004DA002800DC0846221A0DE0002801DD2A
:10176000034600E00B4664339A4205DD002801DDA4
:10177000024600E00A466432BA80A1480322A44C23
:101780004578A248DFF880A2B0F90210AAF1180A41
:101790008B0093FBF2F31293B4F9064001EBD17E78
:1017A00023440F934B005B4293FBF2F31493B0F985
:1017B00000C004EB0C0298180490601AA4EB0C090A
:1017C0000C9009EB01000390A9EB0100119000B20D
:1017D0000190501A0D9000B21590484200EBD0785D
:1017E0000CEBDC701390CCF1000000EBD070029099
:1017F000834803EB090B631890F9A800122D2ED231
:10180000DFE805F02D2E4C5E09FD82A1FC75CBFBB7
:10181000FAF92D2D2DF8AAF80020AAF80290B7F9B0
:1018200004604FF47F7500FB061202F2DC524FF4A5
:10183000FA63AA4201DA2A4602E09A4200DD1A4619
:10184000704C7043A41C401A00F2DC502281A84264
:1018500001DA2B4602E0984200DC03466381DEE1B8
:101860000F9AAAF80020AAF802B0049A6449AAF8CC
:101870000420B7F90430B1F8AA2000FB0320B1F826
:10188000AC20904201DA104604E0B1F8AE10884274
:1018900000DD08465B49891C4881C0E1B7F9044076
:1018A00000FB1433AAF8003000FB049300FB042271
:1018B000AAF80230AAF804200C9A00FB142013E0C6
:1018C000B7F90440039B00FB041100FB1435AAF890
:1018D0000050119D114400FB0455AAF80250AAF8CB
:1018E00004100D9900FB1410AAF8060097E1B7F94F
:1018F0000420514600FB1234AAF80040019C00FB72
:101900000230AAF8024038E1B7F90430129900FB1E
:1019100003440C44AAF8004000FB13B4AAF80240A8
:10192000049C00FB1344AAF804400F9C00FB1344E2
:10193000AAF8064000FB03B4AAF80840149C00FB78
:101940000340104426E0029AB7F90410521002EB4B
:101950006E0600FB014502EB680222442E4400FBA8
:101960001122AAF80060AAF80220139A57465210D2
:1019700002EB6E0602EB68022244354400FB1122A2
:10198000AAF80450AAF806200C9A00FB012200FBDA
:1019900011303A81AAF80A0041E14FEA8C02534221
:1019A00001EBC1020A2592FBF5F94FF0050B93FB01
:1019B000FBF3494201EBC101B7F9046091FBF5F576
:1019C00000FB064703EB090202EB07085919AAF8C6
:1019D00000803944AAF802104FEA8C0C9CFBFBF102
:1019E00001EB090CA44400FB16CC5246AAF804C033
:1019F0000D440FE0B5E07CE03DE015E0F9E0BFE02C
:101A00009804002022010020F8050020A4010020F5
:101A1000B2010020254400FB1655234400FB16307C
:101A2000D5801081C819B5E7B7F90430039C00FBD5
:101A30001345AAF80050119D544600FB0355AAF81F
:101A4000025000FB03155619AAF804600D9E4D4480
:101A500000FB1366AAF80660AAF80850119D11440D
:101A600000FB135500FB1311AAF80A50A1810D9930
:101A700000FB03103AE0CCEBCC050A2695FBF6FE02
:101A8000A1EBC10595FBF6F8BB460EEB0807BBF9C9
:101A90000450C1EBC10100FB054B07EB0B04AAF896
:101AA0000040ACEBCC0494FBF6FC91FBF6F10CEBA4
:101AB00008070CEB010607EB0B04AAF8024006EB43
:101AC0000B047144AAF804405944AAF806100C9972
:101AD00000FB153300FB1511AAF8081000FB159147
:101AE000AAF80A1000FB1520AAF80C30AAF80E007C
:101AF00095E0B7F904B0D44600FB0BF606EB680599
:101B00001544AAF80050029D04EB65056F1A00FB0E
:101B10000B75AAF8025009EB6E0700FB0B75AAF8CB
:101B20000450139D06EB65051D44AAF80650139D4D
:101B300004EB6504611A00FB1B11ACF8081009EBFB
:101B4000680100FB1B11ACF80A10029903EB61015C
:101B500000FB1B11ACF80C1002EB6E0100FB1B101C
:101B6000C4E7B7F90420514600FB0234AAF800404C
:101B7000019C00FB1230AAF8024088801598B3E659
:101B80008848894B90F9B010B3F90220B0F8B850EA
:101B90005143864AB2F902402C44CD1701EB15712E
:101BA00004EB2111B0F8B440A14203DBB0F8B64019
:101BB000A14200DD21467E4C218090F9B110B3F99D
:101BC0000030B2F900205943B0F8BE301344CA17B0
:101BD00001EB1271B0F8BA2003EB2111914201DA46
:101BE000114604E0B0F8BC00814200DD014661808E
:101BF00015E07048AAF80040807A50B16E4A6948F2
:101C0000B2F90020B0F87A100020511A00FB01014F
:101C100002E0002000FB0C0165480180418020208B
:101C2000FFF74FF9E8B35F48002290F8B2108B0736
:101C300007D0614BB0F87A409B89A3EB040363F3B0
:101C40000F02490706D45C49B0F87A30C989C91A2D
:101C500061F31F42B0F8B81011440DB254490D8021
:101C6000B0F8BE3003EB124214B2544A4C80D27822
:101C7000B2B14D4B90F9B020B3F902607243D61760
:101C800002EB167205EB22120A8090F9B120B3F92B
:101C900000305A43D31702EB137204EB22124A802E
:101CA00000E019E0B1F90020B0F8B4309A4203DB4B
:101CB000B0F8B6309A4200DD1A460A80B1F9022027
:101CC000B0F8BA309A4201DA1A4604E0B0F8BC0023
:101CD000824200DD02464A80324E96F8B20000078A
:101CE00012D500252020FFF7ECF800B10225324F75
:101CF000002400BF07EB440001896019C0B203F063
:101D0000FCFE641C042CF5D329490120891E55468C
:101D1000BAF900700B7805E035F91020BA4200DD01
:101D20001746401C9842F7D30024884632E000BF93
:101D3000B6F88800B84205DA35F814103A1A891A4C
:101D400025F8141035F91410B6F88620914201DAFE
:101D5000104602E0814200DC084625F814001648CF
:101D6000B6F87C10B0F90600884207DA1020FFF7B9
:101D7000A8F838B1B6F88A0025F814000D48407864
:101D800018B106E0B6F88600F6E7B6F88A0025F83E
:101D90001400641C98F800008442C9D317B0BDE851
:101DA000F08F000098040020C8000020B20100203D
:101DB0002401002048070020D40100207A070020D9
:101DC0002DE9F74FDFF848A4074690460025DFF8D5
:101DD0003C944FF48056AAF1040B17E000240EE067
:101DE000D9F8001081F00801C9F80010CAF80060A5
:101DF000019803F057FFCBF80060641CE4B2BC42CA
:101E0000EED33C2003F04EFF6D1CEDB24545E5D30B
:101E1000BDE8FE8F2DE9FC5FFE4B002440F2DC5054
:101E2000B3F90610FC4E4FF4FA75814201DA6420D2
:101E30000DE0F948B1F5FA6F90F82E0004DAA1F23E
:101E4000DC52504390FBF5F0C0F16400C0B296F84C
:101E500075B096F876E0B6F87A5081460022B24620
:101E6000EC4840F2E63630F912C0ACEB050000F267
:101E7000F313B34204D8002804DCA5EB0C0001E006
:101E80004FF4FA7080B2022A33D0BBF1000F06D0B3
:101E9000834503D2A0EB0B0080B200E00020642356
:101EA000B0FBF3F3DD4E06EB430736F91380B7F9C9
:101EB0000270A7EB08066FF018077B4300EB830363
:101EC0005E43642396FBF3F3D24E4344223E26F84E
:101ED00012309AF82C3043434FF4FA70B3FBF0F011
:101EE000C0F16400C0B200FB09F06423B0FBF3F062
:101EF00015E0BEF1000F06D0864503D2A0EB0E0020
:101F000080B200E00020C34E223EB0809AF82D300F
:101F100043434FF4FA70B3FBF0F0C0F164000AEBF6
:101F20000208C0B298F80A6064234643B6FBF3F691
:101F3000B84F7E3FBE5498F81E604643B6FBF3F0A0
:101F4000FB1CAC45985406DA03F1590030F8123006
:101F50005B4220F81230521CD2B2032A80D3BAF866
:101F60007C00814201DA014604E04FF4FA639942B1
:101F700000DD194689B2091A4FF47A725143C0F54F
:101F8000FA60B1FBF0F081B26422B1FBF2F0A34B36
:101F90006FF018060C3303EB400533F91030704333
:101FA000B5F9025001EB8000ED1A454395FBF2F0C4
:101FB000DFF86082994EA8F122081844103EA8F874
:101FC0000600707AD146A8F17E05E8B39448B0F9CE
:101FD0000010B5F91A00081A05F02DFF914905F017
:101FE0009EFD914905F0D1FD074606F011FD83469F
:101FF000384607F0C3FA82464746B8F9000005F0B4
:102000001AFF5146009005F08AFD8046B7F902009C
:1020100005F011FF5946019005F081FD414605F09C
:1020200026FD05F016FF80465146019805F077FD24
:1020300082465946009805F072FD514605F069FD4B
:1020400005F007FF388000E001E0A7F802800220D9
:10205000FEF737FF002750B3E878401CC0B20621D6
:10206000B0FBF1F2E87001FB1200B8B902F0B7FD65
:1020700029796A4A01F00703703A491C22F81300D3
:102080002971002032F81010401C2144C0B28CB2DB
:102090000828F7D3E00800F008FE2872287A298C77
:1020A000884203D899F86C10814201D9AF7001E0E1
:1020B0000420A870A87802F083FB5C48534C008889
:1020C00018B10120FEF7E8FE10B95948008820B188
:1020D000206880F00800206014E0F178082011B139
:1020E0004A49091D0860717811B1484908310860F2
:1020F0004FF40060FEF7E5FE20B1707800B10120DA
:1021000002F04FFC8020FEF7DCFE48B1E96BA86AC4
:10211000411A05D44CF250310844E86303F0E0FF63
:10212000A96BA86A411A03D4717BF9B10120F07040
:1021300001F0F8FB1020FEF7AFFE68B1296CA86A29
:10214000411A09D4697A052906D33A490844286412
:10215000206880F0100020603748C16800290ED048
:1021600002B02C48BDE8F05F84380847F77021685A
:1021700081F00801216031490844A863D8E7BDE82F
:10218000FC9F10B5244C204490F86D0003F0C1FC76
:10219000A0F2EE2140F2DD52914201D3B4F87A0070
:1021A00010BD2DE9F0471B4E0024A03E1B4F707957
:1021B000DFF86080401C603F7071A14607F1400568
:1021C000316B20468847727907EBC40102F00302A5
:1021D00021F8120025F814905FF0000035F8143053
:1021E00031F81020401C1A44C0B225F814200428ED
:1021F000F4D335F91400801CC11700EB91708010E6
:1022000025F81400414638F9142019E00C0C01405F
:1022100014080140D4010020980400205807002031
:102220003C020020DB0F494000003443F80100204D
:10223000FA010020F0490200BC07002020A107009D
:10224000D21E904202DA821C21F8142031F91420A7
:10225000D21C904202DD801E28F81400641CE4B2F7
:10226000082CADD3BDE8F0872DE9FC5F002702F014
:10227000EBF908B1FFF795FFDFF8F4A3DFF8F4B34B
:10228000FD4CDAF82810DAF848004FF00005081A7B
:1022900078D444F6206211440820CAF84810FEF7AA
:1022A00010FE08B9FFF77DFF4FF40070FEF709FE3E
:1022B000EF4AA03268B3DFF8C483BAF90C1098F87B
:1022C000816006EB860C8C451BDA6078C8B1B8F9E2
:1022D0007A30002022F81030401CC0B20328F9D315
:1022E000B8F88400D08098F882005346304400EB60
:1022F0008000884201DA65702570D889401CAAF8F0
:102300000E008C4502DA637803B92570491CAAF8DF
:102310000C10DA48B2F906300126B0F87C1091466C
:102320008B426EDAD248DFF854836A3005804580EC
:1023300085802638058045809AF80620521CD2B246
:102340008AF80620B9F90400884205DAB9F90200D2
:10235000884201DA607830B10420FEF7B2FD70B334
:10236000607880B139E0142A0BD1C5484FF47A71F6
:1023700001804FF48070FEF7A4FD002801D002F028
:102380006EF8CDE0E2E1B9F90410B8F87C204846D7
:10239000914222DAB0F90210B8F87E2091421CDD99
:1023A000B9F90000904218DD9AF806105046142939
:1023B00004D1418A21B14582AAF81460B0E00CE052
:1023C000C18B21B10021C18319B1022102E0012199
:1023D000F9E703218AF80010A2E0B8F85810404647
:1023E00081B1A5483230407938B1207828B1667083
:1023F000BBF80010AAF81A1090E06078D0B36570AE
:102400008CE038E0B9F90410B0F87C20CC46914259
:1024100007DB90F88030012B0BD1BCF900309342E0
:1024200007DA62782AB19AF80600142878D1657024
:1024300076E0B0F87E20914207DCBCF900109142B2
:102440006CDD98F88000012868D1B9F9020090424B
:1024500064DA607870B98A48008858B9E07848B181
:102460009AF8061014295BD16670BBF80010AAF820
:102470001A1055E052E0DFF804824846B8F87E2092
:1024800093424DDD63787BBBB0F904308B420CDAAC
:10249000B0F902C08C4508DA9AF8060014280FD16A
:1024A000784B4FF4C8721A800AE093420CDDB0F901
:1024B00002308B4208DA9AF80600142800D1A6737D
:1024C000401C8AF806002BE0B0F90230934203DD8D
:1024D000B8F84000801C04E08B4206DAB8F84000EF
:1024E000801EA8F840000FE01AE0B9F90000904201
:1024F00003DDB8F83E00801C04E088420EDAB8F82C
:102500003E00801EA8F83E000120FEF7AAFB8020B6
:10251000FEF7D7FC20B103F044FE01E08AF8065034
:102520000420FEF7CEFC28B3BAF81E205046322114
:1025300072B1627862B1514AB9F90630B2F87C20C2
:10254000934205DD4C4A323252790AB90182C58381
:10255000494A3232127A32B1C28A438A1A4309D1C5
:10256000AAF8101006E0418A21B1617811B94582BC
:10257000AAF814600020CE4640F2A4680EEB400199
:10258000B1F908C040F214518C4501DA012100E094
:10259000002100EB400901FA09F1ACF21552B2F545
:1025A000C77F01D8012300E0002309F10102934015
:1025B0001943C44501DD012300E0002309F10202B3
:1025C000934019433943401CC0B28FB20428D5D37D
:1025D000DFF8A480294A002008F1320802EB40010C
:1025E000B1F84E10394000D0012108F80010401C0D
:1025F000C0B20E28F2D398F8000038B992F88100E2
:1026000000EB8001BAF90C0081420BDA0120FEF7E1
:1026100043FC38B1207930B91548443005804580F5
:10262000267100E0257198F8050000B9267021791F
:10263000102009B1144901E01349091F0860022064
:10264000FEF72AFC98B198F8010038B3A07970B968
:102650000E480F49A6710068086005487E30C188A1
:102660000C48AAF8181005800B48058018E017E000
:10267000340100203C02002048070020980400207C
:10268000FA010020F8010020140C0140E8000020AD
:10269000EC000020BC000020BA000020FFE7A5717C
:1026A0000420FEF7F9FBD0B198F8020038B1607948
:1026B00030B96671BBF80010FE48018000E065711A
:1026C00098F8090018B1607A10B9667200E0657276
:1026D00098F80D0018B1BBF80010AAF81A101020D5
:1026E000FEF7DAFB48B3E07A38B39AF80900052818
:1026F00025D398F8060050B1E07948B9EE49E67163
:10270000081F01F0E7FE02208AF8010000E0E571F1
:1027100098F8070090B1207A78B9E74A26720C3A07
:1027200002F1100110680860506841F8040F02F1CE
:10273000100001F0CFFE8AF8016000E0257298F8E1
:10274000080008B1A67216E0A57214E09AF9070015
:10275000C21700EB927222F00302821A00F101000C
:102760008AF8070046D0012A4CD0022A52D0032A08
:1027700059D08AF8075003F072FAD04ECAF82800F0
:102780005746318911B1FA6C821A7DD40844F86435
:10279000FEF731FD03F063FAB862F96A411A7981F4
:1027A000F8620420FEF778FB18B3C3481638B0F976
:1027B000041001F145028A2A42D8627992B3BD4AD7
:1027C000BBF8003012889A1A12B212F1B40F02DC70
:1027D00002F5B47212B2B42A02DBA2F5B47212B2DC
:1027E000637B33B1B37C53431E2293FBF2F2891A0D
:1027F000818029E00420FEF74FFB0028BBD000F0C9
:10280000D6FCB8E70220FEF747FB0028B3D000F063
:1028100054FBB0E70220FEF73FFB0028ABD0FEF7E9
:1028200096FDA8E70CE00820FEF736FB0028A2D0B2
:1028300000F05CFDA248A0491E39008888809AE714
:102840009C48BBF8001001800220FEF725FB80B1F8
:10285000A07970B19849B7F918001639B1F9062076
:10286000121A1432282A00D9A571964A12881044E7
:10287000C8801020FEF710FBF0B3E07908B9207A89
:10288000D8B3207BC8B300E06AE15F46BBF9000023
:1028900005F0D1FADFF83082414605F040F906F044
:1028A0006DFE8346B7F9000005F0C5FA414605F014
:1028B00036F906F0ADF882467F4F96F8C700DFF88C
:1028C0000C92443FF0B3B846B7F902003F1DB7F988
:1028D0000210401A01F0BAF896F8C710494288422F
:1028E0000DDBB8F90200B7F90210401A01F0AEF89A
:1028F00096F8C710884201E062E002E004DD084675
:1029000009E001F0C1FD5BE0B8F90200B7F902107F
:10291000401A01F09BF8798808447880B8F90000E3
:10292000B7F90010401A01F091F896F8C710494223
:1029300088420CDBB8F90000B7F90010401A01F02A
:1029400085F800E091E096F8C710884201DD08465E
:1029500006E0B8F90000B7F90010401A01F076F867
:102960003988084400B2388005F065FA594600906D
:1029700005F0D5F88046B7F9020005F05CFA51463B
:10298000019005F0CCF8414605F0C3F8494605F042
:10299000FCF805F05EFA484F5146603F38800098D9
:1029A00005F0BDF880465946019805F0B8F8414653
:1029B00005F05DF8494605F0E8F805F04AFA788038
:1029C000DFF8F4E094F80490AEF1720E0EF13608E0
:1029D000DFF8FCA0002008F1060C08F10C0B00BF8A
:1029E000B9F1000F44D0022842D23349603931F99D
:1029F00010204A3131F91010C2EB4101354A9142A1
:102A000002DB5242914200DD1146334A2B4E6423D1
:102A100032F81020891A06EB4002D28F11440AB214
:102A2000717C514391FBF3F196F8253009B21C46B5
:102A30005B4203EB83038B4203DC04EB84038B4296
:102A400000DA19461C4C503C34F910301A44234B20
:102A50009A4203DB5B429A4200DC13461AB224F826
:102A60001020F37E5A4312134AE0B7F900007BE7C7
:102A70001149114C16393AF9106031F910102A3CFD
:102A800001EB810213010D4A1718BA7A93FBF2F297
:102A9000921B34F9103012B21A44114B9A4202DBE5
:102AA0005B429A4200DD1A4624F8102006F5207693
:102AB00018E000003E020020C80100209804002019
:102AC00020010020BA00002035FA8E3C0000204191
:102AD000F00000200CFEFFFFC8000020F0D8FFFF30
:102AE00080C1FFFFB6F5A06F01D924F8105034F96A
:102AF00010207D2392FBF3F23B7D5A43921112B2D8
:102B00003AF910401EF800305026634393FBF6F369
:102B1000CB1A38F8101028F810403CF810603BF839
:102B20001070611A37442BF810600F442CF8101005
:102B30000C493FB21A44095C7943A2EB6111094A7E
:102B40004B3222F81010401CC0B20328FFF448AFEB
:102B5000FEF7E7FDFEF79CFDBDE8FC5FFEF7C2BD9A
:102B6000BDE8FC9F590100202DE9F843F74CF849D6
:102B700000252F4694F84C20A1F1100003F0BCFB77
:102B800008B101250CE0F24803F055FD08B101271A
:102B900006E0EF4802F0ABFD10B9032003F005F9A1
:102BA000EC4E4FF0000800BF94F8420030B101280D
:102BB00004D0022814D0032828D11FE08DF800800B
:102BC0004FF44870E249ADF802001039684602F04F
:102BD00099F808B10120307094F84200012815D00E
:102BE00065B1DB4994F84C20A1F1100003F084FB9F
:102BF0000220307094F84200022812D0D4481038D5
:102C000003F01BFC10B1032030700AE0307840B9AB
:102C100094F8420010B184F84280C5E70120FEF725
:102C200048F9CB48103003F0E3FD38B9C8481030FC
:102C300002F0FCF810B90220FEF73BF902F008FAA6
:102C400010B90420FEF735F90120FEF725F918B177
:102C5000BF48103800688047BD480068804727B1EA
:102C6000B4F8440003F000FD04E01DB9B4F84400DA
:102C700002F053FDB4F93C00642290FBF2F102FB38
:102C800011000CB205F0D7F8B34904F048FF05462F
:102C9000204605F0D0F8294604F0E9FEAF4904F0DB
:102CA0003EFFAF490860BDE8F88370B50546A74808
:102CB00090F86A0005F0C8F80446284605F0C4F804
:102CC000A84904F02CFFA84904F05FFF214604F056
:102CD00026FF05F0D7F880B270BD70B500252C46F0
:102CE00001F07DFF05440A2002F0DCFF641C202C6B
:102CF000F6D3C5F34F10FFF7D8FF944A022192F89C
:102D00006B3000BF03FB01F4844202D8491C062942
:102D1000F8D39648017092F86C00484394490880B3
:102D200070BD2DE9F047DFF82C92924E874CB9F830
:102D300004200025A2B3864900204FF4C87C343912
:102D4000C846624501D141F8205051F8203036F98B
:102D500010703B4441F8203026F8105004EB40033B
:102D6000401C1D860328ECDB012A14D1086890FB67
:102D7000FCF02086486890FBFCF060868868B8F814
:102D8000081090FBFCF0401AA086E587A4F840509C
:102D90000120FDF766FFB8F80400401EA8F8040003
:102DA0000420FEF78EF800286DD0734BDFF8A4C125
:102DB00067491A880CF11C0C2839ACF11208322A28
:102DC00005D0EAB300209A46322A11D012E0208EB4
:102DD000ACF80000608EACF80200A08EACF80400E5
:102DE000E08FA8F80000B4F84000A8F80200E9E776
:102DF00041F8205051F8203036F910703B4441F82A
:102E0000203026F8105004EB4003401C1D86032898
:102E1000DADB012A19D15948594B05800120188065
:102E2000584B02201870BCF800002086BCF8020045
:102E30006086BCF80400A086B8F80000E08700E0D7
:102E400006E0B8F80200A4F84000521EAAF80020DC
:102E50004D480288012A16D105800A68322092FB6B
:102E6000F0F222864A6892FBF0F26286896891FB52
:102E7000F0F1B9F80800081AA086E587A4F84050D8
:102E80000120FDF7EEFE3088218E401A30807088D8
:102E9000618E401A7080B088A18E401AB080BDE863
:102EA000F08710B52A4C3348103C61688847A16808
:102EB00030488847BDE8104033E770B53348254CAB
:102EC00000682169411A2CD42061214DA078103569
:102ED00040B301282DD0022831D0032821D16869C0
:102EE0008047A869804704F0A6FF294904F04DFEF9
:102EF00004F0FBFF4FF00052264B05F049FE002284
:102F0000254B04F025FF0022244B04F024FF04F09D
:102F1000CDFF234908600020A070A88821690844DB
:102F2000206170BDA8688047A078401CA0702888E8
:102F3000F4E7E8688047A078401CA07070BD28695D
:102F40008047A078401CA0706888E7E798040020BC
:102F5000BC070020F40100208988883C0000204143
:102F6000C40000203333534000F07F45E8010020C7
:102F70005401002008010020440100204A010020E3
:102F80004601002034010020480100205C0100209F
:102F900080E6C547965BC83F0000F03F1AE9504104
:102FA000E40000202DE9F047D24FD34ED34CF888EF
:102FB00030B30025DFF84883A9464FF47A7AF988C0
:102FC000514501D148F8259058F8253034F915C0FD
:102FD0000129634448F8253024F8159026F8159007
:102FE00008D193FBFAF026F8150001220F210A20E0
:102FF000FEF7E6FE6D1C032DE1DBF888401EF8802D
:10300000BC4D002015F1220534F8101036F81020C0
:10301000891A09B224F8101035F91020A2F5487366
:10302000994201DA1A4604E002F54872914200DC46
:103030000A4624F8102025F81020401C0328E3DB62
:103040002DE710B5AE4CAD481C3461688847A168C7
:10305000AA488847BDE81040A4E7A64810B5283024
:1030600002F03FF8A348A749283082880A800288E6
:1030700052424A8040884042888010BD2DE9F04F7E
:1030800085B06020029040F2FE20039040F2C920FB
:10309000049000279C483D46009001F0ECFF954CC1
:1030A00000203C34DFF864A220606060DFF860B28A
:1030B000A0604CE07F1C029801F0EBFF642002F05E
:1030C000F1FDFFF7CAFF0A2002F0ECFD8D4EB6F9C4
:1030D000000004F0B0FE8046039804F0B5FE4146BF
:1030E00004F053FD20F00049B6F9020004F0A3FEFD
:1030F0000646049804F0A8FE3146019004F045FD10
:1031000020F000464146019804F03FFD7F4920F041
:103110000048C94309EB01007E49884217D2564551
:1031200015DD5E4513DAD04511DDD8450FDA6D1C8B
:103130004946206804F09BFC20603146606804F03A
:1031400096FC60604146A06804F091FCA060142FDA
:1031500002D2052DAED301E0052D1BD3284604F085
:1031600073FE05462068009904F0D9FC294604F056
:103170000CFD20606068009904F0D1FC294604F041
:1031800004FD6060A068009904F0C9FC294604F0C1
:10319000FCFC03E04FF07E5020606060A06001F016
:1031A0008EFF54490120487005B0BDE8F08F2DE92D
:1031B000F04759484F4D00686969411A75D457491D
:1031C00008446861FFF749FF4E4CB4F9000004F071
:1031D00032FE05F13C06316804F0A1FC04F039FE32
:1031E00000B220808146B4F9020004F024FE716828
:1031F00004F095FC04F02DFE00B260808246B4F924
:10320000040004F018FEB16804F089FC04F021FE0B
:10321000DFF80C810FFA80FCA4F804C098F80E00C7
:103220000027404A05F12E018B1D88B16869A8610D
:103230005FF0000002EB4006F78634F8106021F8DA
:10324000106023F81060401C0328F3D388F80E7038
:10325000687858B1D68EA9EB06002080168FAAEBAD
:1032600006006080508FACEB0000A080A8690028A9
:103270001BD06E69301A2C4EB04217D22B48026810
:1032800082F008020260002034F9102031F9105059
:10329000AA4201DA21F8102033F91050AA4201DDC8
:1032A00023F81020401C0328EED3F8E50020AF617E
:1032B00031F9104033F910502C4404EBD47402EB74
:1032C00040056410401CEC860328F1D3BDE8F047AC
:1032D0000120FDF7C6BC10B5012003F0F4F808206A
:1032E000FDF7E2FD12490020088010BD104803F0F0
:1032F0003DB90000F40100201A0100200201002065
:10330000A00700201401002059021B3F3333333F34
:103310006666A63F323373005C010020A086010080
:10332000480700209804002080C3C9010C0C01400C
:103330002001002070B5F94C0546C0B2A07002F023
:1033400056FEE079A1784840E071C5F30720A070EF
:1033500002F04DFEE079A1784840E071C5F30740E6
:10336000A07002F044FEE079A1784840E071280E98
:10337000A07002F03CFEE079A1784840E07170BD99
:1033800070B5E64C0546C0B2E07002F030FEE07960
:10339000E1784840E071C5F30720E07002F027FEB5
:1033A000E079E1784840E07170BD10B5044602F064
:1033B0001EFEDA48C1796140C17110BDD74AD848B4
:1033C000117A405C491C1172704700B5FFF7F6FF97
:1033D0000346FFF7F3FF03EB002080B200BD10B5FA
:1033E000FFF7F3FF0446FFF7F0FF04EB004010BDCA
:1033F00070B504460D462420FFF7D7FF4D20FFF798
:10340000D4FF0CB1212000E03E20FFF7CEFFC34CDB
:103410000020E0712846FFF7C8FF607ABDE87040E1
:10342000C3E701460020E3E701460120E0E7BB488F
:10343000C079BAE710B5044603E000BFFFF7B5FF57
:10344000641C20780028F9D110BD02F023BD2DE9BD
:10345000F05FB248B34DDFF8D092407AB34EDFF858
:10346000D0A2DFF8D0B2B44FDFF8D082B44C7328CA
:1034700078D00DDCA0F164000F282BD2DFE800F03B
:1034800091A1FEFDFCFBFAF9F8F7F6F5F4F3F20072
:10349000CC2869D010DCC82822D006DC74287AD069
:1034A000752879D0762815D100E2C92825D0CA28F8
:1034B0003DD0CB280ED149E0D0286ED006DCCD28F7
:1034C0006CD0CE286BD0CF2804D112E0FA2867D078
:1034D000FE2875D00020FFF7A7FFBDE8F05FA6E744
:1034E00000244546FFF771FF25F81400641C082CE2
:1034F000F8D30020FFF795FFEFE7FFF75FFFE872D3
:10350000FFF75CFF89F80000FFF769FF3060FFF705
:1035100066FF7060FFF759FFAAF80000FFF755FF3C
:10352000ABF80000387840F002003870E1E7002383
:10353000FFF744FFE518A872FFF740FF2875FFF773
:103540003DFF5B1CA8770A2BF2D3D2E75FF00005A2
:10355000FFF73BFF04EB45016D1CA1F84E000E2D5B
:10356000F6D3C6E796E1FFE7FFF728FF04F8280F38
:10357000FFF724FF6070FFF721FF2071FFF71EFFA8
:103580006071FFF71BFFA071FFF718FFA070FFF736
:1035900015FFE070ADE76BE16FE1A6E1A9E1ADE1F8
:1035A000AFE10720FFF73DFFD220FFF7FEFE607876
:1035B000FFF7FBFE0020FFF7F8FE4FF0004050E061
:1035C000A3E10A20FFF72DFF5E48008800B2FFF755
:1035D000D7FE01F0C1FF00B2FFF7D2FE0120FDF7D8
:1035E0005BFC04460220FDF757FC44EA400404203B
:1035F000FDF752FC44EA80041020FDF74DFC44EA3C
:10360000C0040820FDF748FC44EA0010FFF7B8FEAC
:103610002879A9796A7840EA41016879800040EA0E
:10362000421001434848C27841EAC201027941EAA6
:103630000211EA7941EA82112A7A41EAC2116A7AD0
:1036400041EA4221AA7A41EA0221827A41EA8221B0
:10365000C27A41EAC221027B407B41EA023141EA5F
:1036600040300CE011E1F5E0E2E0C9E0C0E0B9E093
:10367000A0E08EE074E043E034E025E002E0FFF7F4
:1036800059FE2AE71220FFF7CCFE304D002400BF80
:1036900035F91400FFF774FE641C032CF8D32C4D8D
:1036A000002400BF35F91400FFF76AFE641C032CE8
:1036B000F8D3284D002400BF35F91400FFF760FE51
:1036C000641C032CF8D308E71020FFF7AAFE224D54
:1036D000002400BF35F91400FFF752FE641C082CCB
:1036E000F8D3FAE61020FFF79CFE1C4D002400BF23
:1036F00035F91400FFF744FE641C082CF8D3ECE6FF
:103700001020FFF78EFE00244FEA080535F914005B
:10371000FFF736FE641C082CF8D3DEE640020020DA
:10372000E8070020480700203D010020BC010020E0
:10373000EE010020F0010020E6010020D40100206D
:10374000980400203E0100207A0700200E0100208E
:10375000F00000201401002024010020E0050020DA
:103760000E20FFF75EFEE87AFFF71FFE99F80000D3
:10377000FFF71BFE3068FFF7DDFD7068FFF7DAFD2D
:10378000BAF8000000B2FFF7FBFDBBF8000000B282
:1037900025E00520FFF745FE9D48008800B2FFF7B1
:1037A000EFFD9C48B0F90000FFF7EAFD387800F023
:1037B000010092E00820FFF734FE974D002400BF7F
:1037C00035F91400FFF7DCFD641C022CF8D3934894
:1037D000B0F90000FFF7D4FD9148B0F90000FFF701
:1037E000CFFD7AE60420FFF71CFE8E48006838E71C
:1037F0000320FFF716FE8C480078FFF7D6FD47E060
:103800000720FFF70EFE14F8280FFFF7CEFD6078B3
:10381000FFF7CBFD2079FFF7C8FD6079FFF7C5FD05
:10382000A079FFF7C2FDA078FFF7BFFDE07854E074
:103830001E20FFF7F6FD00256619B07AFFF7B5FDEB
:10384000307DFFF7B2FDB07FFFF7AFFD6D1C0A2D95
:10385000F2D342E61C20FFF7E4FD002504EB45000F
:10386000B0F94E00FFF78CFD6D1C0E2DF6D334E63B
:103870006320FFF7D6FD6D4804E02F20FFF7D1FD50
:103880006A486430FFF7D6FD27E60220FFF7C9FD3E
:103890000020A4E70820FFF7C4FD0024601CC0B28C
:1038A000FFF783FD641C082CF8D316E6FFF786FDAE
:1038B00004460C20FFF7B5FD94B1102C91D11020D7
:1038C000FFF773FD5A4C2068FFF734FD6068FFF77F
:1038D00031FD0020FFF754FD0020FFF766FDFCE5F9
:1038E0000020FFF762FD534CEDE70120FDF7E5F9FD
:1038F000FFE551494FF4C8700880FAE50120A8732C
:10390000F7E50020FDF7ADF9F3E50820FFF789FDA5
:103910004A4D002435F91400FFF732FD641C042CD5
:10392000F8D3DAE570B5464C0025607810B3BDE8F1
:103930007040FCF77CBF00BF02F04CFBA17951B195
:1039400001291CD002291FD0032923D004292CD0FF
:10395000052942D12FE0242803D00021A17149B9C3
:1039600001E00121FAE7232802D0522835D102E0F4
:10397000FCF75DFF31E0012002F03AFA2DE04D281E
:1039800004D10220A07128E03C2801D00020F9E7F2
:103990000320F7E740281FD8607125712572E07178
:1039A0000420A0710120207017E06072E17941408D
:1039B000E1710520E6E721796279914207D2E27947
:1039C0004240E2711F4A5054491C217105E0E179DF
:1039D000814201D1FFF73BFDA57102F0E5FA002815
:1039E000AAD16078002811D102F0DEFA00280DD1AA
:1039F0004FF40060FDF765FA002807D012484078C0
:103A0000002803D0BDE8704000F0DCBF70BD0000AE
:103A1000EA010020EC010020C80000203C02002048
:103A20004E010020E80000203C010020799D0008A4
:103A3000CC010020C4010020F8010020AA010020D0
:103A400040020020E80700204807002044F25061AF
:103A5000884201DDA0EB4100FE49884202DA48F6C7
:103A6000A041084470472DE9F047044640680D46E0
:103A700016469946081A04F0DEF9316804F085F814
:103A80002061A768394604F044F88046F24890F86F
:103A9000C60004F0D9F9F14904F041F801464FF0AD
:103AA0007E5004F072F83668314603F0E0FF0146BC
:103AB000304604F06AF8414604F031F8394603F024
:103AC000D6FF2061C4E901500146D9F8080004F08E
:103AD00026F8BDE8F04704F0BCB970B504460846C6
:103AE00016461D4604F0A7F9696804F018F8316815
:103AF00004F015F8216803F0BAFF01462060E86879
:103B000080F0004004F008FA03D2E86880F000403A
:103B100007E0E968206804F0FFF901D3206801E0BC
:103B2000E8682060BDE8704004F093B970B5CC4CF3
:103B3000D4E90A01401AFFF789FF0028D4E90A01F5
:103B4000A0EB010002DDFFF781FF02E0FFF77EFF3F
:103B5000404241F2941188422ADAD4E90A01401A1B
:103B600004F069F9BF4903F0DAFF0646206B04F060
:103B70006BF90546304605F001FD294603F0CFFFFD
:103B800004F067F900B2B8492081884202DB49425B
:103B9000884200DD0846A16A084448F6A041A063B7
:103BA000884200DD401A002800DA0844A06370BD96
:103BB000A06AFBE72DE9FE4F0646FFF7B7FFA848CE
:103BC00042F22831806B081A04F035F9A54903F058
:103BD000A6FF044604F01CFF0190204605F0CEFC31
:103BE0009F4D009000242435DFF87CB2DFF87CA2E2
:103BF000DFF87C92304604F01EF9029098480E30AF
:103C000030F9140004F017F906465DF82410029804
:103C100003F085FF314603F07CFF04F01AF901B28E
:103C2000944825F81410814202DB4042814200DDB5
:103C3000014604EB84088D4A0AEB880625F8141027
:103C4000603A304600F06DFC884B854A074635F9EE
:103C50001410603B1C323046FFF73FFF834B804A15
:103C6000074435F91410603B1C323046FFF7FBFE69
:103C7000384400B229F81400584501DA584604E0E7
:103C800040F6B832904200DD104629F8140077491A
:103C900030682839641C41F82800022CAEDBBDE8EE
:103CA000FE8F2DE9F05F6E4E00244436A6F1200B06
:103CB000A6F136096D486D4A04EB8407503856F872
:103CC000241000EB8700803A00F02BFC39F8141028
:103CD000D846401A01B265482BF81410283800EB7A
:103CE0008705A0F14802284600F01BFC824638F9FF
:103CF000140056F824105D4B594A0144703B1C32A5
:103D00002846FFF7EAFE594B554A804656F82410DC
:103D1000703B1C322846FFF7A6FE5749884202DB5B
:103D20004942884200DD084639F9141031316229D0
:103D300000D800200AEB080108444B49884202DB06
:103D40004942884200DD0846494921F814004748A5
:103D5000641C00EB870128680860022CAADBBDE820
:103D6000F09F70B50446086819681546401A04F0BB
:103D700062F83B49096A03F0D2FE04F06AF8014692
:103D800037484430416021682A68891A016070BD53
:103D90002DE9F0410E46DDE90685116800681F46F1
:103DA000081A04F048F8044638683168401A04F0EC
:103DB00042F82B49096A03F0B2FE0646014603F0B9
:103DC000AEFE07462146084603F0A9FE394603F039
:103DD0004EFE05F0BFFC294903F0A1FE04F052F8A5
:103DE000C8F8000084F00040314604F0E7FC2449A4
:103DF00003F095FE234903F03AFE04F02AF8286008
:103E0000002803DA48F6A04108442860BDE8F081A4
:103E10002DE9F0471C48124CD0E90065617804F1A7
:103E20003C08B1B14FF07E50E16903F0AEFE82462E
:103E3000D8F80400281A03F0FEFF216A03F06FFE91
:103E4000514603F06CFE04F004F807B204F10E09C9
:103E50001CE03AE0B0B9FFFF98040020DB0FC94036
:103E60004C020020D302373948F4FFFFB808002085
:103E70008401002018FCFFFF30F8FFFF2C7D8E3FEF
:103E8000A00CB34500A00C46BC010020D8F80000EF
:103E9000301A03F0D0FF514603F041FE03F0D9FF82
:103EA00002B204F11800B0F90210394401EBD171EB
:103EB0004910A9F80210B0F900301A4402EBD2728E
:103EC0005210A9F800204180028001206070C8E9EA
:103ED0000065BDE8F08710B5044603F0ACFF002C88
:103EE00001DC80F00040FE4903F019FE04F090FD73
:103EF000FC49086210BD70B5034600200246054625
:103F000011E02E2C04D1521C00290FD054181D553D
:103F10009C5C00EB80004000A4F13006092E01D823
:103F200030382044521C9C5C002CEAD170BD2DE935
:103F3000F041002580462E462F46044603F0F8FC4B
:103F4000016800E0641C2078085C2028FAD0404614
:103F500009E01DB105EB85025206150E10F8012B84
:103F6000303D2A44D5B2221A022AF2DC09E01EB101
:103F700006EB86025206160E10F8012B303E324434
:103F8000D6B28442F3D820782E280ED1641C0020AB
:103F900007EB8702570022788B5C202B02D1303F41
:103FA0001744641C401C0428F2DBCF48062146431A
:103FB00007EBC70000EB071006EB8000B0FBF1F049
:103FC000CA494D4300EBC51020E72DE9F047002713
:103FD000C44C05463E464FF00109242814D0214622
:103FE000C348C9782C2D13D02A2D11D022460D2D6F
:103FF000527973D00A2D71D00F2902D24554491C31
:10400000E170002A6BD084E0A670E670267180E033
:104010004654A178B046324629B1A279012A21D06E
:10402000022A5DD06BE0A2710178472967D14178FF
:10403000502964D18178472902D0522909D05EE005
:10404000C17847295BD10079412858D184F806907E
:1040500055E0C1784D2952D1007943284FD1022033
:10406000A0714CE0A34E02290CD003290ED00429E4
:1040700013D0052915D006291AD0072921D00929DE
:1040800026D03CE09A48FFF752FF04E0007853281E
:1040900035D130684042306031E09548FFF747FF46
:1040A00004E0007857282AD170684042706026E00A
:1040B0000078302801D9012000E000208E49C87224
:1040C0001DE000218A48FFF716FF8C49087016E0B2
:1040D00000218748FFF70FFF89490FE026E015E030
:1040E00007290CD101218248FFF705FF41F2184151
:1040F00048434FF47A71B0FBF1F082490880A07810
:10410000401CA07084F803802A2D0CD020796840D0
:104110002071A07910B17C4A82F800900FB101287B
:1041200000D00020D5E684F80590F2E772B1804611
:10413000007800F028FA050198F8010000F023FA51
:1041400028442179C0B2884200D101276671E0E796
:104150002DE9FF5FC0B2FFF738FF00287ED06B4823
:1041600000220178012911D0012101706248C17A31
:10417000002973D06149097805296FD341785D4DD5
:10418000584C824621B1027B2AB112E00270EDE761
:104190008AF80C200DE061B101218AF80C105C490D
:1041A000286808606A684A60FFF795FE59480088E9
:1041B000A08120780521401CB0FBF1F201FB120226
:1041C0008E4655492270002091F900904FEA050B68
:1041D00044495BF820305C31424C41F820304F4973
:1041E0006C3493FBF1F144F82010404C00EB800557
:1041F00064424C4303EBC41342F2107493FBF4F497
:104200001FFA84F8374C343424F81080384CB83412
:1042100004EB8505334C55F82260543454F8207073
:1042200045F82230BE1B334444F8203093FBFEF3A4
:104230002E4C614303EBC1112A4B6433B9F1010FDA
:1042400043F8201006D1A8F10208B8F5797F01D80B
:104250004BF82010401C0228BADB00E09BE001F084
:1042600013FD204C6169401A03F0EEFD2C4903F068
:104270008CFCE06101F008FD6061E0694FF07E5167
:10428000884200DB0846E06103A902A8204BCDE983
:1042900000011B1D5D461A1F291D1648FFF778FDFA
:1042A00002986426B0FBF6F01E49088003981E4968
:1042B00090FBF6F00880FFF7ABFD9AF8081019B9EB
:1042C0009AF80700002866D00649283101F1080055
:1042D00000F11C073B1DCDE900013A46291D25E0F0
:1042E00050E0EF304C02002040420F002D31010021
:1042F00028080020BC010020480700203D010020C4
:10430000EE010020F0010020E7010020E60100207E
:10431000C40100203C020020350100208096980056
:1043200000007A44EA010020EC0100209D48FFF7DC
:104330002FFD2B1D9B4A391D3846FFF712FD9A4D64
:1043400095F90000012828D0022824D1974F012197
:10435000B7F9CC0000F0F1F8FFF72CFC97F8C80093
:10436000934A18B1A06B90FBF6F01080B7F8C40028
:10437000216B88420BD2D4E90A01401AFFF766FB91
:10438000002800DC404242F21071884203DD012027
:104390002870A0891080BDE8FF9FFFF782FCFAE734
:1043A0002DE9F047814C0E34207803F04DFDDFF805
:1043B0000492494603F0E9FB7F4D2860A07A03F0A0
:1043C00043FD494603F0E1FB7C4EEE606860607897
:1043D00003F03AFD7A4F394603F0D7FB10352860D9
:1043E000E07A03F031FD494603F0CFFB6860607D61
:1043F00003F02AFDDFF8CC81414603F0C6FBC5E996
:104400000206A07803F020FD394603F0BEFB10350C
:104410002860207B03F018FD494603F0B6FB686076
:10442000A07D03F011FD414603F0AFFBC5E9020694
:104430004FE510B50446FFF7B3FF6349204601F08E
:10444000EDFD4FF4FA7001F02DFC60480078002873
:1044500004D0BDE810401020FCF726BD10BD5C481C
:10446000C17A00290FD05B49097805290BD34D4942
:10447000594A0B681360496851605849584A09887D
:1044800091810121017370472DE9F05FDFF82891D8
:10449000002409F13009534FDFF84C81264609F119
:1044A000280A09F1500B00BF27F8146004EB8405BB
:1044B00028F8146009EB850000F06EF80AEB85001F
:1044C00000F06AF80BEB850000F066F8641C022C23
:1044D000EADB44E47CB5424C02684C342260096853
:1044E00061600068FFF7F7FCA4F1240101F1080006
:1044F0002C4ECDE90001231D2246311D3046FFF729
:1045000047FC374D331D3246A86AA863211D20465B
:10451000FFF727FCA86AE8622448B0F8CA0068815F
:104520007CBD10B50846144603F085FC216803F0F5
:10453000F6FABDE8104003F08CBC70B5284C226B35
:1045400041B1B0EB520F00D3500800B200280CDC90
:1045500000200AE0904200D31046144900B2B1F89E
:10456000CA10814200DB084600B2B4F90A50A842E2
:1045700008DD1049E06903F0D2FA03F06AFC284430
:1045800000B2608170BD3038C0B2092801D9C01FA7
:10459000C0B200F00F0070470021016041608160EF
:1045A00070470000BC010020350100209804002065
:1045B0003E0200200000C842380800200000FA44F3
:1045C0000000204100007A4451410008E70100202A
:1045D000480700203D010020C40100203C020020CB
:1045E0004C020020680100208401002070B5364C88
:1045F00001260546667001F032FBA168421AC4E943
:10460000020241F288300021824200D9A1702F4A73
:10461000A07815540F2802D0401CA07070BD2C4803
:104620002670018070BD2B48032190F87820264821
:1046300012B1C170072101E00222C2700171264946
:104640004FF4E13001F0EABC1F4800787047F0B544
:104650001D4A1E4B11781C3BE1B11679D578DFF865
:104660006CE003210EEB010717F8014CEC4004F05D
:104670000F04072C08D21EF801C017F8017C374040
:104680000CEB072743F82470891CC9B21029E9D321
:10469000002111700F4907280FD252786AB10D4AD4
:1046A00091F87810104490F86D0053F8200039B15B
:1046B0004FF4777101EB500004E0B1F87A00F0BDDF
:1046C00000F5777080B2F0BDC00200202409002000
:1046D0004001002098040020ED4500082DE9F0413C
:1046E0007E4C0746012520782E0380B901F0CCFAD4
:1046F000A1683231884207D379482570066001F0FD
:10470000C3FAA060BDE8F08120780028FAD001F05B
:10471000BBFAA16839448842F4D300202070704865
:10472000001F066001F0B0FAA0606E48017809B180
:10473000491E01706570E5E7F8B5684D8DF8000019
:104740008DF801108DF802208DF80330A8791DF83E
:10475000001044292FD04C292BD04D2927D04E2989
:104760002CD032240026032806D274B12046FFF74D
:10477000B5FFA879032808D301F086FAA968001BC1
:10478000884202D95748AE7106706878012801D076
:10479000002C0BD1A879032801D2401CA8715049E4
:1047A0006E70091F2E704FF480500860F8BD6424AD
:1047B000D8E7C824D6E74FF4FA64D3E70024D1E75A
:1047C0002DE9F047DFF820A10546444C9AF80A008D
:1047D0004FF00109002610B184F8029000E0A670A5
:1047E0004FF40070FCF76DFB404F18B3404941484F
:1047F0004FF0020891F88130B0F9000003EB83021A
:1048000082420FDA97F801C0BCF1000F0AD084F899
:10481000049091F88210194401EB8101814201DA80
:1048200084F80480824203DA797809B984F8048034
:1048300000B926711020FCF72FFB40B19AF8061042
:1048400011B99AF8070008B1F87AA8B1E670207992
:10485000022814D0012817D0E078012817D0A078BA
:10486000012817D0042D19D0022D1ED0012D1ED0E5
:10487000607901281ED022E084F80390E7E74E22F9
:10488000442311464C200DE04D234C2208E04D23DB
:104890004E2201E04D235322532102E044234D22B6
:1048A0004D215320BDE8F04746E7442305E044236B
:1048B0004E22F5E7787810B14E234D22ECE70948F7
:1048C000007818B1BDE8F047322007E704492670A8
:1048D000091F4FF480500860BDE8F087D002002027
:1048E00014080140340100207A0700204807002006
:1048F000980400204001002070B5132000F0F3F868
:10490000834C2068002800DC4042824D90FBF5F08B
:1049100000B200F0F2F81B2000F0E5F82068002853
:1049200000DC404290FBF5F042F2107690FBF6F18D
:1049300006FB110000B200F0E0F8232000F0D3F8ED
:104940002068002801DA532000E04E2000F0D5F85E
:10495000122000F0C8F86068002800DC404290FB9C
:10496000F5F000B200F0C9F81A2000F0BCF8606859
:10497000002800DC404290FBF5F090FBF6F106FBCE
:10498000110000B200F0B9F8222000F0ACF8606825
:10499000002801DA572000E04520BDE8704000F013
:1049A000ACB870B55C4D04462878844209D014B187
:1049B0004FF4165002E05948D0F8D000FEF745FDFC
:1049C0002C7070BD2DE9F04701F05EF9524D696819
:1049D000401AC8287DD301F057F968606878504FB5
:1049E000401CDFF84081DFF840916870002400BF70
:1049F00004F12400C0B200F076F8388803F024FAFD
:104A0000064638F9140003F016FA314603F0BDF8F3
:104A1000494603F084F803F01CFA00B200F06DF888
:104A2000641CE4B2032CE3D3102000F05CF83F4C8C
:104A30006426206890FBF6F000B200F05EF82120BA
:104A400000F051F8206890FBF6F106FB110000B26F
:104A500000F053F8022000F046F835480A21B0F97A
:104A6000000090FBF1F000B200F047F85E2001F08A
:104A7000BEFA68780521B0FBF1F201FB120040B9E3
:104A80001020FCF709FA20B1FFF736FF5E2001F095
:104A9000AEFA6878192824D10020687001F0F4F883
:104AA0004FF47A71B0FBF1F43C25B4FBF5F6B6FB9C
:104AB000F5F005FB1067172000F015F8380200B27A
:104AC00000F01BF8182000F00EF805FB164000B2AD
:104AD00000E006E000F011F8BDE8F0475E2001F0CC
:104AE00086BABDE8F08710B504465E2001F07FFA73
:104AF0002046BDE8104001F07ABA10B50446C0B2B5
:104B000001F075FAC4F30720BDE8104001F06FBA58
:104B1000BC010020A0860100DC02002098040020D7
:104B2000FC0100200E01002000007A44E800002073
:104B30005001002070B52B4E90B0304602F046F880
:104B400029480090294801A90024012531C12802E3
:104B50000494CDE9054080000790202008900002D1
:104B6000CDE909046946304602F09DF8012130463E
:104B700002F0B6F88DF830400B948DF831504FF4B8
:104B80006020CDE90D04184C8DF83C504C3C0BA92D
:104B9000204601F087FF032301220421204601F073
:104BA000D6FF0121204601F0A6FF0121204601F099
:104BB00098FF204601F0A9FF204601F0ABFF002836
:104BC000FAD1204601F0ADFF204601F0AFFF0028EA
:104BD000FAD10121204601F0B0FF10B070BD0348AA
:104BE00000887047080002404C240140E402002085
:104BF00070472DE9FC47DFF84891054699F8000019
:104C0000C0B300263746B0463446641CE4B26B4657
:104C100008223221532000F061FC9DF800009DF82D
:104C20000110202C00EB012000B206449DF8020088
:104C30009DF8031000EB012000B207449DF804002A
:104C40009DF8051000EB012001B29DF80700884493
:104C500000F07F0001D20028D7D196FBF4F0288025
:104C600097FBF4F0688098FBF4F0A88089F8014085
:104C7000BDE8FC87FFE76B4606223221532000F097
:104C80002DFC9DF800009DF8011000EB012028800C
:104C90009DF802009DF8031000EB012068809DF84C
:104CA00004009DF8051000EB0120A880E0E72448EF
:104CB00010B500784FF0080200284FF02D014FF09A
:104CC00053000ED000F004FC0A223121532000F0E2
:104CD000FFFB0C222C21532000F0FAFB90223821FC
:104CE00008E000F0F5FB0A223121532000F0F0FB30
:104CF0000A222C21532000F0EBFB124940F209104C
:104D0000088010BD38B5054600200C468DF800001F
:104D100001466B460122532000F0E0FB18B19DF8DC
:104D20000000E52801D0002038BD0549287808702A
:104D300005482060054860600548A060012038BD36
:104D4000E6020020FC010020AF4C0008F34B0008F5
:104D5000F14B000810B54FF48044204602F01AF8D9
:104D6000012805D1204602F023F8B049012008703F
:104D700010BD30B4AD4AAE4891884389B0F91440B3
:104D8000C91A03895943C913B0F912300C44DB0224
:104D900093FBF4F31944C161906830BC00F0C7B8CC
:104DA00038B5A24C207810B96088401C60806B46F2
:104DB0000322F621772000F091FB9DF800009DF87A
:104DC0000110000440EA01209DF8021008439849B0
:104DD000B1F92010C1F10801C840A06038BD944865
:104DE0003421008C01EB80109049C2B20020087081
:104DF000F421772000F06CBB38B58C4C207810B9CA
:104E00006088401C60806B460222F621772000F00B
:104E100065FBBDF8000040BAA08038BD8349002082
:104E20002E220870F421772000F052BB2DE9F043C8
:104E3000DFF8F891044685B099F8010018B1012017
:104E400005B0BDE8F0834FF40058ADF80C800220A7
:104E50008DF80E001020774E8DF80F00454603A9FF
:104E6000304602F011FC4FF48047ADF80C7004207E
:104E70008DF80F0003A9304602F006FC35610E21C3
:104E8000022002F08FFC00208DF808000820019716
:104E90008DF8090001278DF80A7001A801F044FF80
:104EA00028208DF810000F208DF811008DF81200C9
:104EB0008DF8137004A801F0C2FD142000F0F2FE7A
:104EC0006B460122D021772000F008FB584D9DF859
:104ED00000000321E8752984552803D0C6F8148002
:104EE0000020ADE76B460122D121772000F0F6FAD1
:104EF0009DF8000000F00F0129760009687600F0A7
:104F00005EF889F8017041F2F810208046F2905066
:104F1000608041F28830A0804748A0604748E06048
:104F200047482061474860614748A06187E770B5FE
:104F30003F49CA69B1F90E30A2F57A6202FB02F666
:104F400034136343DC12B1F90230534304EBE3231F
:104F5000B1F9004003EB84030C8CA3409B1C9D1013
:104F6000B1F90430361353435A13B1F90C30C988E0
:104F7000734302EB2342921C921002F5004251430C
:104F8000C90B401B4CF25032E2405043B0F1004F8D
:104F900003D24000B0FBF1F002E0B0FBF1F04000C2
:104FA0000112494340F6DE325143284A0914424374
:104FB00001EB224101F6CF6100EB211070BD00B57D
:104FC00087B06B461622AA21772000F087FABDF839
:104FD000000041BA16480180BDF8021049BA41806C
:104FE000BDF8041049BA8180BDF8061049BAC180E5
:104FF000BDF8081049BA0181BDF80A1049BA4181CB
:10500000BDF80C1049BA8181BDF80E1049BAC181B2
:10501000BDF8101049BA0182BDF8121049BA418298
:10502000BDF8141049BA818207B000BDE802002023
:1050300034090020001001401D4E0008F94D000801
:10504000DF4D0008A14D0008734D000843E3FFFF4A
:1050500008B500208DF800006B4601220A211E20B1
:1050600000F03CFA18B19DF80000482801D000205B
:1050700008BD012008BD10B5642000F013FE7822A1
:1050800000211E2000F024FABDE81040322000F07C
:1050900009BE10B50446792200211E2000F018FA3E
:1050A000322000F0FFFD224601211E2000F010FA00
:1050B00001220221BDE810401E2000F009BA10B5FF
:1050C000782200211E2000F003FA202201211E2058
:1050D00000F0FEF900220221BDE810401E2000F081
:1050E000F7B91CB504466B46062203211E2000F0CA
:1050F000F5F9BDF8000040BA2080BDF8020040BAC2
:105100006080BDF8040040BAA0801CBD30B587B0F7
:1051100005464FF44060ADF8140002208DF81600EB
:105120001C208DF8170005A9FE4802F0ADFAFE4CD0
:10513000E56000F014FAE06801F040FE684601F016
:10514000A8FE00224FF44071E06801F0D8FE00256F
:10515000ADF804504BF6FF70ADF806004FF48040F8
:10516000ADF80C00F14800900121E06801F09FFECD
:105170006946E06801F035FE4FF4A06001F05AFC8A
:1051800022208DF810008DF811508DF8125001205A
:105190008DF8130004A801F052FC21208DF81000B6
:1051A0008DF8115004A801F04AFC07B030BD70B56D
:1051B000DD4CE068858A15F4706F01D00121217003
:1051C00015F4E06F24D0018B00224FF4806101F0D0
:1051D00096FEA8051CD4E0680188890518D40188CA
:1051E000C9050CD50188C905FCD4012101F073FE65
:1051F000E06801888905FCD4FFF788FF08E00121F9
:1052000001F069FE00224FF44071E06801F077FE82
:10521000E068818A21F4706181820020207170BD74
:10522000C5E72DE9F041C04CE068818A4FF00105E7
:10523000C9B2CA074FF0000627D0018821F40061E7
:105240000180012101F051FEE670607A20B16078A2
:1052500060B9A079FF2809D061790022E06801F0E7
:105260005BFEA079FF280FD0FF20B8E06570E079E1
:10527000022804D1E068018841F40061018061796D
:105280000122E06801F048FEC9E08A074FF4806718
:1052900034D5BFF3508FE079012810D1607A70B116
:1052A000607860B10021E06801F01FFEBFF3508F0D
:1052B000E068018B012101F00EFEA5701CE0E068A2
:1052C000008BBFF3508FE07902280DD1607A58B17E
:1052D000607848B10021E06801F007FE93E03946AC
:1052E000E06801F00CFE9AE0E079032804D1607ACE
:1052F00010B16078002874D10122F0E74A0753D535
:10530000A570627A88494978CAB3C9B3E17902299C
:105310001FD9002101F0E9FDE06801F0FAFD94F9E0
:10532000032063699854521CE2700121E06801F087
:10533000D2FDA570E06801F0ECFD94F903106269FC
:105340005054491CE17001223946E06801F0D7FD54
:1053500025E0012101F0BFFDE06801F0DAFD94F9DC
:10536000031062695054491CE170E06801F0D1FDFE
:1053700094F9031062695054891CE1700FE000E059
:1053800000E009B9217A31B1012101F0A4FDE078F2
:10539000401CE07003E0012101F093FD6570E068BE
:1053A0000188C905FCD43AE04A061BD501F0B1FDDD
:1053B00094F9031062695054491C48B2E070E179D5
:1053C000C01C814204D100223946E06801F097FDFB
:1053D000E17994F90300814221D100F10100E070EC
:1053E0001DE010E009061AD594F90320511C4BB2B8
:1053F0000BD02569A95CE37001F089FDE07994F98F
:10540000031088420BD1002269E7E370A17901F013
:105410007EFD607A0028F6D1E0790028F3D094F977
:105420000310E079401C814209D16670A07828B150
:1054300000224FF44071E06801F061FD2671BDE883
:10544000F081EEE6B3E6ECE67FB5374C400047F27C
:1054500030556071A1710121217200266672C4F875
:1054600010D0C4F814D06846E27121712670102A59
:1054700002D9002004B070BD002103E05E5C4654F8
:10548000491CC9B29142F9D3E068818889050ED4DC
:105490000188C90505D401888905FCD4012101F0E2
:1054A00010FD01224FF44071E06801F028FD2079E1
:1054B00010B16D1EFBD104E01DB1207880F0010019
:1054C000D8E76089401C6081E068FFF71FFED0E7E5
:1054D00007B502AB0122FFF7B7FF0EBD70B5124C46
:1054E0004FEA400047F230556071A17100202072F0
:1054F0000121617263612361E27121712070E068B2
:105500008188890516D40188C90505D401888905D3
:10551000FCD4012101F0D5FC01224FF44071E06878
:1055200006E00000000C0140F4020020801A060092
:1055300001F0E5FC207910B16D1EFBD104E01DB136
:10554000207880F0010070BD6089401C6081E068B7
:10555000FFF7DCFD002070BD2F48408970472DE922
:10556000F8434FF44067ADF800704FF002088DF833
:1055700002801420294C8DF803006946204602F071
:1055800083F83946204602F0E0F80025261502E0AF
:105590000A2000F07CFB3146204602F0CFF80028BC
:1055A000F6D03146204602F0D2F80A2000F06FFB18
:1055B0003146204602F0C9F80A2000F068FB6D1C55
:1055C000EDB2082DE7D34FF400652946204602F0DE
:1055D000BEF80A2000F05BFB3146204602F0B7F827
:1055E0000A2000F054FB3146204602F0AEF80A20B3
:1055F00000F04DFB2946204602F0A7F8ADF80070F8
:105600008DF802801C208DF803006946204602F0C8
:105610003BF8BDE8F8830000F4020020000C0140D4
:1056200038B504466B4602221B216820FFF756FF5F
:10563000BDF8000043F2903140BA08444FF48C7139
:10564000B0FBF1F02330208038BDB0F90010CA174C
:1056500001EB927189100180B0F90210CA1701EBB9
:10566000927189104180B0F904104942CA1701EBC8
:1056700092718910818070471CB504466B460622E2
:105680001D216820FFF72AFFBDF8000040BA2080E6
:10569000BDF8020040BA6080BDF8040040BAA080A6
:1056A0001CBD10B5192000F0FDFA0022152168205C
:1056B000FFF70EFF10B9032000F077FB28481621F2
:1056C000007840F018026820FFF702FF002217213F
:1056D0006820FFF7FDFE01223D216820FFF7F8FE5C
:1056E00001223E21BDE810406820FFF7F1BE10B551
:1056F0000446192000F0D6FA002215216820FFF791
:10570000E7FE002808D01748206017486060174857
:10571000A0601748E060012010BD1149622817D031
:1057200006DC0A281AD0142816D02A2809D111E03C
:10573000BC2804D0B0F5807F03D1002000E0012018
:1057400008700878162140F018026820FFF7C0BEE4
:105750000220F5E70320F3E70420F1E70520EFE757
:105760000C030020A3560008795600084B56000889
:105770002156000870B51646FF4B00EB800203EB84
:105780008205FE4A02EB0014206800F0C6F9D4E955
:105790000101002200F047FA217B3246206800F028
:1057A000D2F9A07B18B10121206801F080FE01210F
:1057B000206801F072FE207B30B1042807D0082851
:1057C0000AD00C2806D10AE02068343001E02068B5
:1057D00038306860284670BD20683C30F9E72068A2
:1057E0004030F6E7F8B517460E46E34A00EB800175
:1057F00002EB8105E14901EB00144FF6FF712068CF
:1058000000F08BF9D4E90101012200F00CFA217BB0
:105810000022206800F0EFF90121206801F03DFE30
:10582000607B8DF8000000208DF8010001208DF8CC
:1058300002008DF80300684601F001F92E60AF7296
:10584000207B30B1042808D008280DD00C2809D1BD
:105850000EE001220221206802E0012204212068DA
:1058600001F030FE2846F8BD012208212068F7E744
:10587000012210212068F3E770B5C14C02212046B7
:1058800001F04BFEBC4D012814D01021204601F040
:1058900044FE01281AD109261021204601F048FEB5
:1058A000204601F037FED5F8B42001463046BDE869
:1058B0007040104708260221204601F039FE20469C
:1058C00001F022FE0146D5F8A020EFE770BD70B5CB
:1058D0000C460646022101F020FEA74D012823D0E8
:1058E0000421304601F019FE012826D00821304657
:1058F00001F013FE01282AD01021304601F00DFEE0
:1059000001282ED1E41C64B21021304601F010FEB3
:10591000304601F0FFFD014604EB840055F82020DD
:10592000E0B2BDE87040104764B20221304601F099
:10593000FFFD304601F0E8FDEDE7641C64B2042190
:10594000304601F0F5FD304601F0E0FDE3E7A41C30
:1059500064B20821304601F0EBFD304601F0D8FD7D
:10596000D9E770BD00214FF08040B0E704218548A1
:10597000ADE70A218448AAE7804A30B5083A0023F7
:105980009088D0809180081A81B240F68C208142A4
:1059900001D9D37030BD7948A1F2EF24083840F224
:1059A000DB55C078AC4204D2082802D2774C24F8E8
:1059B0001010401CD0707648038030BD6E4A00EB5A
:1059C000800370B502EB83026C4BD47A03EB0013B7
:1059D00018681B7B84B1D18194896C4D091B11829D
:1059E000947A25F814100024D4722246194600F047
:1059F00002F96748048070BD91810121D172BDE830
:105A000070400222194600F0F6B82DE9F04706462C
:105A10000020317901B10220717801B1401C574951
:105A2000DFF87081E031002451F82070A1F1E80521
:105A30004FF47A793A5D02F00F0002F0F001FF2A8C
:105A40004CD011F0300F02D0327802B90021B27878
:105A500022B1082801D0092800D18021F2781AB19A
:105A6000021F032A00D88021CA0605D500224A4910
:105A7000FFF7B8FE082008E08A0608D5AA7847494B
:105A8000FFF7B0FEA87800F10100A87023E04A06F5
:105A900010D5F288B8FBF2F189B24A46FFF76AFEE8
:105AA00001463A4A2878103242F8201000F10100ED
:105AB000287010E009060ED53289B8FBF2F189B2E0
:105AC0004A46FFF757FE0146304A6878403242F8AE
:105AD0002010401C6870641C0E2CABDB0020BDE85D
:105AE000F087264A083A1278904205D2274A1032A7
:105AF00052F82000406801807047204A083A5278E6
:105B0000904205D2214A403252F82000406801807C
:105B100070471E4931F8100070473EB505460C46E7
:105B2000684601F09FFC4720ADF80000641E00208D
:105B3000ADF80440ADF80600ADF80200694628460D
:105B400001F070FA3EBD7FB506460C461546684624
:105B500001F091FC7020ADF800000120ADF80200CA
:105B60000020ADF804000220ADF80800C001ADF837
:105B70000650ADF80C0013E058090020180300206F
:105B8000002C01400004004000080040700A002082
:105B90004001002040420F0079590008BD5900081B
:105BA00074B1042C15D0082C1CD00C2C07D16946DC
:105BB000304601F017FB0821304601F09EFC7FBD06
:105BC0006946304601F067FA0821304601F082FC50
:105BD0007FBD6946304601F093FA0821304601F056
:105BE0007FFC7FBD6946304601F0C4FA082130468B
:105BF00001F07DFC7FBDFEB506460C4615466846A5
:105C000001F043FC0120ADF804000021ADF8004094
:105C1000ADF80610ADF80810ADF8025069463046F0
:105C200001F088FBFEBDF8B506460C4615466846F1
:105C300001F07CFDADF800400DB1282000E01820F7
:105C40008DF8030002208DF802006946304601F00D
:105C50001BFDF8BD6B484168491C4160704710B599
:105C600068494FF0E02348689A694C68A042FAD12D
:105C70006549891A4822B1FBF2F100EB4002C2EB00
:105C8000C01001EBC00010BD5E484068704730B5E1
:105C90000546FFF7E4FF0446FFF7E1FF001BA842BB
:105CA000FAD330BD30B504464FF47A7502E0284689
:105CB000FFF7EDFF641EFAD230BD2DE9F0418CB044
:105CC0001822524901A801F060FE03270121504823
:105CD00001F087F9012144F61D2001F079F9012135
:105CE000084601F06CF901F08EF94FF6FF70ADF83F
:105CF000000000268DF803606946464801F0C4FCA8
:105D00006946454801F0C0FC6946444801F0BCFCC6
:105D10000121434801F01DFD002401AD4FF00208B0
:105D200005EBC4008188ADF800108DF80280807901
:105D30008DF8030055F83400694601F0A5FC641C99
:105D4000BC42EDD3344808211030016010210160BD
:105D5000304980141031086007A801F0EBF8314990
:105D60000798B0FBF1F0274908602F484FF47A718B
:105D70000068B0FBF1F0B0F1807F0BD220F07F41E2
:105D80004FF0E020491E4161284AF02111708661E0
:105D900007210161FEF7CEFE2548FFF7B7F9642021
:105DA000FFF780FF0CB0BDE8F0811B4A10211432D0
:105DB00011600821121F1160044640F2DB10154FDC
:105DC000151F44434E021437A7F1040C286880F0D5
:105DD00010002860286880F008002860A01EFFF7E7
:105DE00061FF3E601920FFF75DFFCCF80060EDE732
:105DF00010B111490F4808600C4910481739086064
:105E0000704700000804002040190100449E00086B
:105E10000700400000080140000C01400010014054
:105E20000002300040420F004C04002023ED00E04F
:105E300000580040EFBEADDEF04F00200400FA0530
:105E4000A148A04A41685318A04A136583688B4251
:105E500003D9591A9164436004E0C1F580719164DB
:105E60000021416099480121443000F039BF10B54C
:105E70004FF4005000F04AFF94480021443000F0F5
:105E80002FFF9148001D03C8814202D0BDE8104099
:105E9000D6E710BD2DE9F04192B004464FF40070F2
:105EA000ADF83C0002208DF83E001820884D8DF89A
:105EB0003F000FA9284601F0E7FB2815ADF83C008C
:105EC00048208DF83F000FA9284601F0DDFB0E2089
:105ED0008DF8400001218DF841108DF842108DF8A9
:105EE000431010A800F0ABFD0B940024ADF8344033
:105EF0000C20DFF8E081ADF83040ADF83600ADF8A9
:105F00003240ADF838400BA9404601F015FB6F4F09
:105F10005837384600F05AFEA81408F104050095D9
:105F2000CDE909046C48CDE9010480260494CDE94B
:105F30000564A81503902020CDE90740694638463E
:105F400000F0B1FE0121384600F0CAFE01224021D6
:105F5000404601F06BFB384600F0D5FE5A495B4FD6
:105F600044370860384600F031FE1020029000955A
:105F70000494CDE90564079469463846089400F016
:105F800092FE01220221384600F0B5FE4F4884649B
:105F900001228021404601F049FB0121404601F0E9
:105FA00023FB12B0BDE8F081484810B5583000F02E
:105FB000AAFE45490968884201D0012010BD002091
:105FC00010BD4148D0E90110814201D10120704744
:105FD000002070473C49404B0A68C2F58070185C4D
:105FE000521E0A6002D14FF480720A607047364A2E
:105FF000344B91685854491CC8B290603348406C87
:10600000C00700D11CE7704710B5044602E0641CCD
:10601000FFF7EDFF20780028F9D110BD70B50D46CF
:106020000646012186B0480400F0DBFF26208DF8EB
:10603000100001208DF8110002218DF812108DF84A
:10604000130004A800F0FBFC0820ADF814000424A1
:106050008DF8174005A91E4801F016FB0020ADF889
:106060000800ADF80A40ADF804001C4CADF806007D
:10607000ADF80C0000966946204601F05DFA012259
:1060800040F22551204601F0B9FA0121204601F0E5
:10609000ABFA0D48C56006B070BD70B50F4D40F24B
:1060A0002551284601F0CEFA01280AD1064CE068B5
:1060B000002806D0284601F0C1FAE168BDE870402A
:1060C000084770BDD00B00201004002000000240E3
:1060D0000008014000380140D00A00200044004080
:1060E000FEB5384C0125207878B1012822D002284D
:1060F0001FD164208DF8000033488DF80150002630
:106100004078A0B38DF8025043E07A208DF800006B
:106110002E486B460222B0F90000FF21C0F1B40006
:1061200000EBD07040108DF801006D20FFF78CF966
:106130002570FEBD264979208DF80000B1F90000D8
:106140000A2290FBF2F010F15A0301D5002003E07F
:106150005A30B42800DDB4208DF80100B1F90200F6
:1061600090FBF2F010F15A0102D5002004E00EE09D
:106170005A30B42800DDB4208DF802006B460322AB
:10618000FF216D20FFF760F902202070FEBD8DF821
:1061900002606B460322FF216D20FFF755F9267040
:1061A000FEBD08B56B208DF800000A208DF80100B7
:1061B0008DF802006B460322FF216D20FFF744F9A2
:1061C00008BD000020040020480700203C020020F9
:1061D000C8000020B0F90010CA1701EB92718910B5
:1061E0000180B0F90210CA1701EB92718910418049
:1061F000B0F904104942CA1701EB927189108180ED
:1062000070471CB504466B46062243216820FFF701
:1062100065F9BDF8000040BA2080BDF8020040BA20
:106220006080BDF8040040BAA0801CBD10B580227B
:106230006B216820FFF74CF90520FFF733FD0022A2
:1062400019216820FFF744F903226B216820FFF72A
:106250003FF9022237216820FFF73AF903221A2179
:106260006820FFF735F918221B216820FFF730F965
:106270003848007814280CD015280AD0542808D0A3
:10628000552806D010221C21BDE810406820FFF7D9
:106290001FB90822F7E7B0F90210B0F90020CB17B8
:1062A00001EB5371C91001805142CA1701EB5271C1
:1062B000C9104180B0F90410CA1701EB5271C9101E
:1062C000818070471CB504466B4606223B2168203E
:1062D000FFF704F9BDF8000040BA2080BDF80200C5
:1062E00040BA6080BDF8040040BAA0801CBD1A49C5
:1062F00040F2FF3008807047F8B504460D46164658
:106300002320FFF7CFFC6B46012275216820FFF7A1
:10631000E5F8002804D09DF80000682801D000208E
:10632000F8BD1EB10B495520087005E0094B01224C
:106330000C216820FFF7D2F8084820600848606008
:106340000848A06008482860084868600848A860B5
:106350000120F8BD21040020FC010020EF620008AC
:10636000C5620008976200082D62000803620008F9
:10637000D5610008B0F900104942CA1701EB9271CB
:1063800089100180B0F902104942CA1701EB9271DD
:1063900089104180B0F90410CA1701EB927189107D
:1063A000818070471CB504466B46062201211C20E3
:1063B000FFF794F8BDF8000040BA00B22080BDF8A5
:1063C0000210801049BA09B26180BDF80420208013
:1063D00052BA881012B260809010A0801CBD10B517
:1063E00000222A211C20FFF773F802220E211C2014
:1063F000FFF76EF803220F211C20FFF769F8122225
:106400002B211C20FFF764F802222C211C20FFF70F
:106410005FF801222D211C20FFF75AF800222E21BF
:106420001C20FFF755F805222A211C20FFF750F801
:1064300011494FF48070088010BD38B50446002023
:106440008DF800006B4601220D211C20FFF746F855
:1064500028B19DF800002A2803D01A2801D0002076
:1064600038BD06492160064961600649A1600649B8
:106470000870012038BD0000FC010020DF63000827
:10648000A5630008756300082204002010B5444C81
:106490004448A18801F052F918B1FFF7E0FBA06071
:1064A0000AE0FFF7DCFBA168884205D9401A3B21CE
:1064B00090FBF1F061690880E068BDE8104000F0F1
:1064C00077BCE3E7E2E7FEB50125354C022110B1C8
:1064D000012810D109E04FF4807060804000A08056
:1064E000E06009202070172004E06580A180E16051
:1064F0002570072060706088ADF8000010268DF8C8
:106500000360284F8DF802106946384601F0BCF848
:10651000A088ADF8000004208DF8030069463846D5
:1065200001F0B2F82178012001F03CF9E06800F0B8
:106530003FFCE068019000208DF808008DF80960AC
:106540008DF80A5001A800F0EFFB94F9010000F06B
:106550001F018D4040094FF0E02101EB8000C0F8A1
:106560000051FFF791FB3C382061FEBD70B5054638
:10657000FFF78AFB0A4C21693C3188420FD3C4E9FA
:106580000405084D6188284601F0DFF80B20FFF76D
:106590007EFB61882846BDE8704001F0D8B870BD28
:1065A00024040020000C0140B0F900104942CA1731
:1065B00001EB927189100180B0F90210CA1701EB4A
:1065C000927189104180B0F904104942CA1701EB59
:1065D00092718910818070471CB504466B46062273
:1065E000A8216820FEF77AFFBDF8000040BA60805D
:1065F000BDF8020040BA2080BDF8040040BAA08077
:106600001CBD10B56420FFF74DFBF022232168204C
:10661000FEF75EFF10B90320FFF7C7FB0520FFF769
:1066200041FB1E4820210078BDE8104040F00F02D9
:106630006820FEF74DBF38B504461920FFF732FB3E
:106640006B4601220F216820FEF748FF9DF80000ED
:10665000D32801D0002038BD114820601148606067
:106660001148A060012038BD0C49202806D03628EA
:1066700006D04E280DD05D2804D10CE0002000E0AB
:10668000402008700878202140F00F026820FEF7B3
:106690001FBF8020F5E7C020F3E700003C04002086
:1066A00003660008D9650008A96500082DE9F04FC8
:1066B000DFF87CA2DFF87CE24FF00008BAF80A109D
:1066C000DEF80400BAF80830A0EB0122A3FB026751
:1066D000BAF80400D517040408FB027003FB050395
:1066E000F00940EA436014EB000BBAF80640BAF830
:1066F0000200A4FB027C4FEAC03548EBE3114046A0
:1067000000FB02C34FEAE27604FB06334FEA17248C
:1067100044EA036415EB040C40EB2320BAF80C3078
:106720004446A3FB02674FEAE27504FB027203FBD7
:1067300005224FEA422343EAD6524FF4FA63D218B5
:10674000C146B2F5FA6F17DAA2F5FA635B4303EBC1
:1067500083034FEA63084FEAA309774B9A420BDAA7
:1067600002F2DC525243C2EBC203984402EB4203F2
:1067700003EBC20309EB6309BBEB080261EBE871B1
:10678000BCEB0903DEF808404FF00005A4FB0367EB
:1067900005FB037360EBE97004FB00304FEA5653CE
:1067A00043EAC0234FEA60509A1A60EB01004104AB
:1067B00041EAD230BDE8F08F10B500F070F85D49C5
:1067C000886010BD5B48012200784030C1B277205C
:1067D000FEF77EBE10B500F062F85649486010BD65
:1067E0005448012200785030C1B27720FEF770BEC5
:1067F0002DE9FE4305464FF40054ADF80040022059
:106800008DF8020010204D4E8DF803006946304689
:1068100000F03AFF74610A20FFF744FA02AB01224C
:10682000A0217720FEF75AFE002823D001221E2146
:106830007720FEF74DFE4FF42F60FFF728FA002473
:10684000DFF8EC802646A02707EB4400C1B201AB7D
:10685000022277200196FEF741FEBDF8040040BAFF
:1068600028F81400641C082CEEDB314800F029F8ED
:1068700010B10020BDE8FE8342F2107028806880CD
:106880004FF47A60A8802E48A8602E48E8602E4811
:1068900028612E4868612E48A8610120EAE708B502
:1068A0006B46032200217720FEF718FE9DF80000BA
:1068B0009DF80110000440EA01209DF802100843F1
:1068C00008BDF0B5C289002102F47F4502F00F0433
:1068D0000123C5814FEA010230F8126006B100239E
:1068E000521C082AF8DB4FF0FF36F3B90022D30719
:1068F00022F00103C35A02D0DBB2594001E081EA21
:10690000132108230F0401D581F4C05149005B1EF7
:10691000002BF7DC521C102AE9DB2543C581C1F3AB
:106920000330844201D10020F0BD3046F0BD0000AC
:10693000D00C00204004002024FAFFFF001001408A
:10694000E1670008D5670008C5670008B967000857
:10695000AD660008324810B5016841F001010160E0
:106960004168304A1140416001682F4A114001607E
:10697000016821F480210160416821F4FE01416039
:106980004FF41F01816000F005F828494FF00060C6
:10699000086010BD22480021026842F48032026083
:1069A0004FF4A063026801F1010112F4003F01D12C
:1069B0009942F7D10168890330D51D490A6842F030
:1069C00010020A600A6822F003020A600A6842F0B4
:1069D00002020A604168416041684160416841F4D7
:1069E00080614160416821F47C114160416841F45B
:1069F000E8114160016841F080710160016889011E
:106A0000FCD5416821F003014160416841F0020179
:106A100041604168C1F381010229FAD17047000049
:106A2000001002400000FFF8FFFFF6FE08ED00E056
:106A3000002002401849084318490860704770B5A3
:106A40000F21C478027801234FF0E026DCB1134C0B
:106A5000246804F4E064C4F5E064250AC5F1040484
:106A6000E9404578A54084780C402C4321010C4C2A
:106A70001155007800F01F018B40400906EB8000A3
:106A8000C0F8003170BD02F01F008340500906EBD2
:106A90008000C0F8803170BD0000FA050CED00E008
:106AA00000E400E010B54268464B0C791A400B68D0
:106AB00042EA0422134343608368434A1340D1E906
:106AC000024222434C7943EA44031A438260C26A79
:106AD000097C22F47002491EC9B242EA0151C16226
:106AE00010BD0029816802D041F0010101E021F0D0
:106AF0000101816070470029816802D041F48071F2
:106B000001E021F4807181607047816841F00801E3
:106B100081607047014600208968090700D501207F
:106B20007047816841F00401816070470146002090
:106B30008968490700D5012070470029816802D083
:106B400041F4A00101E021F4A0018160704770B51B
:106B5000072509290AD9C468A1F10A0606EB4606E9
:106B6000B540AC43B3401C43C46007E0046901EB8B
:106B70004106B540AC43B3401C4304611F23072AC0
:106B800009D2446B521E02EB820293409C43914017
:106B90000C43446370BD0D2A09D2046BD21F02EB73
:106BA000820293409C4391400C43046370BDC46ACD
:106BB0000D3A02EB820293409C4391400C43C46225
:106BC00070BD0000FFFEF0FFFDF7F1FF01684FF61A
:106BD000FE72114001600021016041608160C1606E
:106BE0004F494F4A0839904203D1486840F00F009E
:106BF00006E04B4A1432904204D1486840F0F0005D
:106C000048607047464A2832904203D1486840F4B1
:106C10007060F5E7424A3C32904203D1486840F444
:106C20007040EDE73E4A5032904203D1486840F44C
:106C30007020E5E73A4A6432904203D1486840F454
:106C40007000DDE7364A7832904203D1486840F060
:106C50007060D5E7334A111F904203D1086840F0B5
:106C60000F0006E02F4A1432904204D1086840F029
:106C7000F000086070472B4A2832904203D1086820
:106C800040F47060F5E7274A3C32904203D108682F
:106C900040F47040EDE7234A50329042EAD1086850
:106CA00040F47020E5E730B5036847F6F07293438F
:106CB0000C6A8A682243D1E904452C4322438C693B
:106CC0002243CC6922434C6A22438C6A22431A43F2
:106CD0000260CA6842600A6882604968C16030BD6B
:106CE0000029016802D041F0010102E04FF6FE7276
:106CF000114001607047002A026801D00A4300E099
:106D00008A4302607047406880B27047C10003D573
:106D10000449091F086070470149083948607047F5
:106D2000080002400804024030B523498379026814
:106D300053B30B6893430B600A1D13680468A343A5
:106D4000136002790A4413680468234313601A4AE3
:106D5000083213680468A3431360131D1C68056898
:106D6000AC431C604479102C05D021440A680068AB
:106D700002430A6030BD116804682143116019683C
:106D800000680143196030BD0079084401689143EF
:106D9000016030BD084A014600201268064B0A40D7
:106DA00014331B680B4202D0002A00D00120704728
:106DB0000149143108607047000401405A4910B578
:106DC00088424FF0010101D14C0501E04FF48004ED
:106DD000204600F00FF92046BDE81040002100F0E9
:106DE00009B970B50446808886B00D4620F03F068C
:106DF000684600F09FF84D490298B0FBF1F189B266
:106E00000E43A680228822F001022280484B2A6885
:106E10009A421CD85200B0FBF2F080B2042800D293
:106E20000420491C2184A083208840F00100208098
:106E300021884FF6F5300140A8886A89104308433D
:106E40002080A88929890843208106B070BDEB887D
:106E5000A3F53F46FF3E05D102EB4202B0FBF2F044
:106E600080B208E002EBC20303EB0212B0FBF2F0C7
:106E700080B240F48040020501D140F001004FF49F
:106E8000967251434FF47A72B1FBF2F140F4004034
:106E9000C7E741F288310160002181804BF6FF7223
:106EA000C280018141814FF4804181817047002976
:106EB000018802D041F0010101E021F001010180CF
:106EC00070470029018802D041F4807101E021F46B
:106ED0008071018070470029018802D041F400715F
:106EE00001E021F40071018070470029018802D07F
:106EF00041F4806101E021F4806101807047002A43
:106F0000828801D00A4300E08A4382807047018270
:106F10007047008AC0B2704712B141F0010101E030
:106F200001F0FE01018270470054004040420F0012
:106F3000A0860100374910B54A6812F00C03364AA2
:106F400003D0042B01D0082B26D002604A68334BB3
:106F500002F0F00212099C5C0268E24042604C6858
:106F600004F4E064240A1C5D22FA04F484604C6892
:106F700004F460544FEAD4241B5D22FA03F2C26089
:106F80004968264B01F440414FEA91311B1F595C7F
:106F9000B2FBF1F1016110BD4A684B6802F4701256
:106FA0004FF0020413F4803F04EB924202D04B688E
:106FB0009B0301D51A4B00E0174B5A43C5E7154A0E
:106FC0000029516901D0014300E0814351617047BC
:106FD000104A0029916901D0014300E08143916189
:106FE00070470C4A0029D16901D0014300E0814378
:106FF000D1617047074A0029116901D0014300E0BF
:107000008143116170470348416A41F080714162D8
:10701000704700000010024000127A006404002053
:1070200000093D0030B50288F84BF94C98420DD06C
:10703000A0420BD0B0F1804F08D0F64DA84205D049
:10704000F54DA84202D0F54DA84203D122F07005BB
:107050004A882A43F24DA84206D0F24DA84203D0F6
:1070600022F44075CA882A4302808A8882850A8869
:10707000028598420AD0A04208D0EB4A904205D03F
:10708000EA4A904202D0EA4A904201D1097A018646
:107090000121818230BD30B5028C22F001020284D0
:1070A000028C8388048B22F0020224F073050C8882
:1070B0002C430D8915434A882A43D44DA8420BD04E
:1070C000D34DA84208D0D84DA84205D0D74DA842EC
:1070D00002D0D74DA8420DD122F008054A8923F4E9
:1070E00040732A4322F004058A882A438D891D4370
:1070F000CB892B4383800483C9888186028430BD79
:1071000030B5028C22F010020284028C8388048B3A
:1071100022F0200224F4E6450C88240645EA1444B3
:107120000D892D0542EA15454A88120545EA1242A5
:10713000B64DA84202D0B64DA84215D122F0800526
:107140004A8923F44063120545EA124222F04005C1
:107150008A88120545EA12428D89AD0443EA154535
:10716000CB899B0445EA134383800483C988018744
:10717000028430BD30B5028C22F480720284028C0D
:107180008388848B22F4007224F073050C882C43CE
:107190000D892D0642EA15454A88120645EA124233
:1071A0009A4DA84202D09A4DA84215D122F400650A
:1071B0004A8923F44053120645EA124222F48065BC
:1071C0008A88120645EA12428D892D0543EA154543
:1071D000CB891B0545EA134383808483C988818753
:1071E000028430BD30B5028C22F480520284038CBC
:1071F0008288848B24F4E6450C88240645EA1444EE
:1072000023F400550B891B0745EA13434D882D07CE
:1072100043EA15457D4B984202D07D4B984205D1FB
:1072200022F480438A89920543EA12428280848351
:10723000C988A0F84010058430BD828B22F44062DA
:107240008283828B42EA012282837047828B22F002
:107250000C028283828B0A4382837047028B22F462
:1072600040620283028B42EA01220283704770B5BA
:10727000048C24F010040484068B048C26F47346DA
:107280001B0746EA1343120643EA12420D055F4B01
:107290002D0C98420ED05E4B98420BD0B0F1804F2F
:1072A00008D05C4B984205D05B4B984202D05B4BB8
:1072B000984205D124F02001294341F0100104E057
:1072C00024F0A0030B4343F010010283018470BD3E
:1072D000028B22F00C020283028B0A430283704766
:1072E00030B5048C24F001040484058B048C1B0548
:1072F00042EA134325F0F305444A2B4390420ED053
:10730000434A90420BD0B0F1804F08D0414A90429E
:1073100005D0414A904202D0404A904202D124F026
:10732000020201E024F00A020A4342F00101038351
:10733000018430BD2DE9F05F0D4604460E883348C8
:10734000DFF8CCC0DFF8CCA0DFF8CCE04988AA8811
:107350002B894FF0804B3EB3042E2DD0082E268C67
:1073600032D026F480562684B4F81C90268C0F0761
:107370004FEA1748120629F473471B0747EA1242DF
:1073800042EA134384420AD0644508D05C4506D0E3
:10739000544504D0744502D02048844256D126F486
:1073A000005040EA080054E02046FFF799FFE988C2
:1073B0002046BDE8F05F8BE72046FFF758FFE988DD
:1073C0002046BDE8F05F49E726F480762684A78B47
:1073D000268C1B0527F0F30742EA13434FEA0168A6
:1073E0003B434FEA184884420AD0644508D05C45C4
:1073F00006D0544504D0744502D00848844219D1BF
:1074000026F4007040EA080017E00000002C01405C
:10741000003401400004004000080040000C00401F
:1074200000100040001400400040014000440140B2
:107430000048014026F42060084340F48070A38394
:107440002084E9882046BDE8F05FFFE626F402408C
:10745000084340F48050A3832084E9882046BDE897
:10746000F05FEAE64FF6FF71818000210180C18064
:107470004180017270470021018041808180C1807C
:10748000018141818181C18170470021018041805A
:1074900001228280C180018170470029018802D0C9
:1074A00041F0010101E021F0010101807047002954
:1074B00030F8441F02D041F4004101E0C1F30E0155
:1074C00001807047002A828901D00A4300E08A4384
:1074D00082817047028B22F008020A4302837047C0
:1074E000028B22F4006242EA012101837047828B01
:1074F00022F008020A4382837047828B22F40062E2
:1075000042EA012181837047808E7047008F704767
:10751000808F7047B0F840007047038A002280894E
:107520000B4200EA010001D000B101221046704771
:10753000C94301827047000030B50446008A85B017
:107540000D464CF6FF710840E98801432182A1896C
:107550004EF6F3100140A8882A8910436A890A432D
:107560001043A081A08A4FF6FF410840A98901433A
:10757000A1826846FFF7DEFC4248844201D10398AD
:1075800000E00298A1890904002900EBC00101EB89
:107590000010296802DA4FEA410101E04FEA810157
:1075A000B0FBF1F06422B0FBF2F14FEA01114FEAB7
:1075B00011136FF018056B4300EB8300A3891D04C2
:1075C0004FF0320306D503EBC000B0FBF2F000F041
:1075D000070005E003EB0010B0FBF2F000F00F0035
:1075E0000843208105B030BD0029818902D041F4D3
:1075F000005101E021F400518181704710B5C1F3C1
:10760000421301F01F040121A140012B07D0022BDE
:1076100007D01430002A026805D00A4304E00C3079
:10762000F8E71030F6E78A43026010BD002A828A2C
:1076300001D00A4300E08A43828270478088C0F309
:107640000800704770B501F01F0601220025C1F344
:10765000421302FA06F4012B0FD0022B0FD0838ABB
:107660004FEA11210088234202FA01F200EA0200E7
:1076700001D000B10125284670BD8389F0E7038A57
:10768000EEE70000003801402DE9F041CB780025FD
:1076900003F00F02DB0601D58B781A430B884FF0FD
:1076A0000F0813F0FF0F4FF0010C1CD0D0F8004072
:1076B0000E880CFA05F31E409E4210D1AF0008FA66
:1076C00007F624EA060602FA07F43443CE78282E99
:1076D00002D0482E02D002E0436100E003616D1C3D
:1076E000082DE5D304600B88FF2B1DD944680025C5
:1076F00005F108060CFA06F30E881E409E420FD1D3
:10770000AF0008FA07F624EA060602FA07F4344343
:10771000CE78282E00D14361CE78482E00D1036167
:107720006D1C082DE4D34460BDE8F0814FF6FF7175
:107730000180022181700421C1707047024600203F
:1077400092680A4200D00120704701617047416190
:107750007047F0B51C4C002801DAE36900E063686B
:10776000420D120185B2C0F301579540C0F30346A4
:10777000032F05D0C2020AD50322B240934307E08B
:1077800023F07062636823F07063636002E0AB43D0
:1077900043F0706201B12A43002801DAE261F0BDD2
:1077A0006260F0BD10B58A0721F003040649130F8B
:1077B00021440F228C689A4094438C608A689840D8
:1077C00002438A6010BD000000000140374836497E
:1077D00041603749416070473448016941F0800198
:1077E0000161704731490420CA68D20701D00120E5
:1077F0007047CA68520701D502207047C968C90698
:10780000FBD50320704700B50346FFF7EBFF02E00E
:10781000FFF7E8FF5B1E012803D0002B00D10520F5
:1078200000BD002BF4D1FAE770B505464FF43026C1
:107830003046FFF7E8FF042811D11C4C206940F0C6
:10784000020020616561206940F0400020613046FF
:10785000FFF7D9FF216941F6FD721140216170BD2A
:10786000F0B505464FF4005C0E466046FFF7CBFFCF
:10787000042814D10D4C206940F0010020612E80B5
:107880006046FFF7C0FF41F6FE77042804D1300CB4
:1078900068806046FFF7B7FF216939402161F0BD7C
:1078A0000249C8607047000023016745002002407C
:1078B000AB89EFCD14481549026800608A4203D0B5
:1078C0001348804713480047134E4FF009003060BB
:1078D0001248016821F07061016041020160104CA2
:1078E000182020600F49104808601048D0F800D0D8
:1078F00040680047FEE7FEE7FEE7FEE7FEE7FEE73B
:10790000FEE7FEE7FEE7FEE7F04F0020EFBEADDE4C
:1079100055690008ED0000081810024004000140FD
:10792000140C0140000C01404434434400F0FF1F9C
:10793000004870476C9F0008A0F16101192900D828
:10794000203870472DE9F05F83460F46154699466B
:107950004FF0FF36DDF828A011E0A819441009FB0C
:10796000047080460146584652469047002802D08F
:1079700004DA254603E04046BDE8F09F2646A5EB25
:1079800006000128E9DC0020F6E740EA01039B0736
:1079900003D009E008C9121F08C0042AFAD203E084
:1079A00011F8013B00F8013B521EF9D27047D2B2E8
:1079B00001E000F8012B491EFBD270470022F6E7D8
:1079C00010B504460846114602462046FFF7EFFF71
:1079D000204610BD30B50EE003460A4601E05B1CB0
:1079E000521C1C781578AC4201D1002CF7D115F04F
:1079F000FF0F04D0401C0278002AEDD1002030BDDA
:107A0000CAB20178914203D009B1401CF9E70020C5
:107A100070470146002000E0401C0A5C002AFBD1B0
:107A200070472DE9F041054600200E469046044679
:107A300000E0641C44450BD2285D00F0A8FA07461C
:107A4000305D00F0A4FA381A02D1295D0029F0D186
:107A5000BDE8F08170B5064600F086FD0468054675
:107A60000A220021304600F098FA2C6070BDF0B474
:107A700080EA0102D20F4300B3EB410F02D203466A
:107A8000084619464B0042D0C30DDDB2C1F3C754BE
:107A90002C1B202C35DAC1F3160141F4000502B18C
:107AA0006D42C4F1200605FA06F125412844B3EBE6
:107AB000D05F23D0C2B1012CA0EBC35009DCF0BCD5
:107AC0004FF0004202EAC35200F50000DBB200F0C2
:107AD000A5BA400000F1807000EBC350A0F18070A7
:107AE00040EAD170490009E0490841EAC071A0EBC1
:107AF000C35000F50000400800EBC350F0BC00F09C
:107B000084BA5142012303EB4101801AF6E7F0BC2D
:107B1000704781F00041AAE780F00040A7E780EAC3
:107B2000010210B502F00042400026D04B0023D0E5
:107B30004FEA106101EB1361C0F35600C3F3560323
:107B400040F4000043F40003A0FB0330A1F17F01E7
:107B50004FEA00401C0401D000F1010050EA13403C
:107B600001D44000491EC3B20C0604EBD010401CE7
:107B70004008802B02D003E0002010BD20F001005F
:107B8000002900DA0020104310BD80EA010202F053
:107B9000004330B430F0004221F0004015D0A0B1D5
:107BA000C0F3C755C2F3C754C2F31601C0F31600A1
:107BB000651B41F4000140F400007D35814201D392
:107BC0006D1C00E04900002D02DA30BC0020704737
:107BD0004FF400020024814201D3091A14435208D1
:107BE0004FEA4101F7D151B1814202D14FF000413A
:107BF00005E002D24FF0010101E06FF0010104EB5A
:107C0000C55030BC184400F000BA2DE9FE4F0746BD
:107C100081EA0300C00F0E46019021F0004123F0DD
:107C20000044B81AA14105D23846314617461E46CF
:107C30000B46024623F00040104304D1384631463B
:107C400003B0BDE8F08F350DC5F30A00C3F30A5148
:107C50000290401A0090402868DAC3F3130040F401
:107C6000801B0198924620B10023D2EB030A63EBFC
:107C70000B0B00985946C0F14002504600F056F9EF
:107C800080460C4650465946009A00F06EF9C019DD
:107C90007141EF1785EA11533B4340D0019A52B32B
:107CA000009A012A11DC0022801A4FF0004361EB98
:107CB000055103EA05538018CDE9002341F58011F1
:107CC0004246234600F03DFABAE72E050025401B48
:107CD00061EB0601401941F5801200185241281845
:107CE000A6F5001343EB020140EAD470294318EBD8
:107CF0000808644113E064084FEA38084FF00002B6
:107D000044EAC0744FEA0553801A61EB03018018FE
:107D100041F5801149084FEA300080185941424628
:107D2000234603B0BDE8F04F00F0FEB901980122F0
:107D300040000023D0EB020263EBE07301984FEAAE
:107D4000E074381A66EB0401EBE783F000435CE76C
:107D500081F0004159E72DE9FE4F81EA030421F04B
:107D6000004504F0004423F000414FF0000A009465
:107D700050EA050302D052EA010304D10020014673
:107D800003B0BDE8F08FC1F30A53C5F30A541C4495
:107D9000A0FB02B3C5F3130545F4801CC1F3130126
:107DA00041F480180CFB023300FB083EA4F2F334CC
:107DB000810A930A41EA8C5143EA88530194A1FB5A
:107DC00003474FEA9C2505FB03734FEA982601FB06
:107DD00006373D05260545EA1435BBEB06016EEB7B
:107DE0000503850E920E45EA8C1542EA8812A5FB22
:107DF0000206261E67EB00070C0D44EA0334A419A3
:107E000047EB1350C1F313064FF0000319464FEA36
:107E1000033343EA165343EA0403019CE5FB0201E2
:107E2000A4F10C040294009C4FEA0632CDE900A4B0
:107E300000F087F9A4E7C10F80EAE0700844CA07A0
:107E40009623002100F0EAB896230022114600F0A4
:107E5000E5B800F0004220F00040C10DC0F316006C
:107E600040F400007F2901DA00207047962903DCE6
:107E7000C1F19601C84001E096398840002AF4D04B
:107E80004042704720F00040C10DC0F3160040F49E
:107E900000007F2901DA00207047962903DCC1F138
:107EA0009601C840704796398840704770B5C1F355
:107EB0000A5201F000450024C1F3130140F2FF33E0
:107EC00041F480119A4201DA002070BD40F2334340
:107ED0009A42A2F2334203DC524200F036F800E04C
:107EE00090402C43F1D0404270BD00F0004230F091
:107EF00000400DD0C10D01F5607142EA0151002230
:107F0000C0F31600520742EAD002400711437047FF
:107F10000020014670470000002801DBC0F100404E
:107F2000002901DBC1F1004188427047202A04DBAF
:107F3000203A00FA02F1002070479140C2F120037C
:107F400020FA03F3194390407047202A04DB203ABB
:107F500021FA02F00021704721FA02F3D040C2F169
:107F600020029140084319467047202A06DBCB17B0
:107F7000203A41FA02F043EAE071704741FA02F315
:107F8000D040C2F120029140084319467047A0F149
:107F90004101192900D8203070472DE9F0470F46DC
:107FA000914680460446002614F8015B2DB1FFF788
:107FB000BFFC0068405DC007F6D12B2D02D02D2DEF
:107FC00018D0641E4A463946204600F0C9F927B148
:107FD0003968A14201D1C7F8008071054FF0020451
:107FE0000BD54042002803DD00F0BEFA0460A00774
:107FF000BDE8F08746F48066E4E70028F8DA00F090
:10800000B3FA04606FF00040F2E70029A8BF7047A0
:10801000401C490008BF20F00100704710B4B0FABE
:1080200080FC00FA0CF050EA010404BF10BC704759
:1080300049B1CCF1200421FA04F411FA0CF118BF73
:10804000012121430843A3EB0C01CB1D0106000ACB
:10805000002BBEBF002010BC704700EBC350104483
:108060000029A4BF10BC7047401C490008BF20F085
:10807000010010BC7047420005D0C0F3C752524205
:10808000914201DC0020704700EBC1507047F0B412
:10809000002802DCF0BC00207047C0F3C751C0F3D9
:1080A000160040F40000CA0701D14000491E3F22DB
:1080B00002EB6105002211464FF4000626FA01F397
:1080C0001344D418844201D8001B1A464000491CAE
:1080D0001729F3DD5100814202D24FF0FF3100E059
:1080E000002102EBC550F0BCFFF78FBF10B5410077
:1080F0000CD0C0F3C751962908DC7E2909DC06DBC9
:10810000410204D000F0004040F07E5010BD00203D
:1081100010BDC1F19604C4F1200100FA01F1E04064
:10812000FFF773FFA04010BD10B5002B08DA401C0C
:1081300041F1000192185B411A4301D120F0010086
:1081400010BD2DE9F04D92469B4611B1B1FA81F276
:1081500002E0B0FA80F220329046FFF7E7FE0646D2
:108160000F4640EA0A0041EA0B0152465B460843CB
:1081700003D130463946BDE8F08D194652EA010078
:1081800015D0C8F140025046FFF7DFFE04460D4609
:10819000504659464246FFF7C9FE084301D0012028
:1081A00000E00020044345EAE07526432F430A9887
:1081B0004FEAD625A0EB08000A304FEA46534FF0AD
:1081C000000245EA47554FEAD72402D50020014670
:1081D000D1E7010550196141DDE908450019694100
:1081E000BDE8F04DA0E72DE9F04D81EA030404F06D
:1081F000004B21F0004714464FF0000A23F00041E5
:1082000050EA070220D054EA01021DD0C1F30A55FA
:108210000246C1F31300C7F30A56C7F3130340F431
:10822000801143F48013A6EB0508101BD64608F214
:10823000FD3873EB010002D308F1010801E0921848
:108240005B41B8F1000F03DA00200146BDE8F08D74
:1082500000204FF48015064607460EE0B2EB040CF2
:1082600073EB010C04D3121B064363EB01032F4392
:108270006D084FEA300092185B4150EA050CEDD1D1
:1082800052EA030012D082EA040083EA010528437F
:1082900003D100224FF0004308E0101B8B4102D2B3
:1082A0000122002302E06FF0010253101AEB0600D6
:1082B00047EB085110EB0A0041EB0B01BDE8F04D14
:1082C000FFF732BF70B521F0004303430CD0C1F378
:1082D0000A540026D4EB060566EB0603D417AD1A44
:1082E000A34102DB0020014670BD001C41EB02519E
:1082F00070BD0EB5C10F80EAE0700844CA070021C6
:1083000040F233438DE80E000A460B46FFF719FF93
:1083100003B000BD30B5002904DB4FF000444042FB
:1083200064EB0101002B04DB4FF00044524264EB8C
:108330000303994208BF904230BD0000064C074D30
:1083400006E0E06840F0010394E807009847103425
:10835000AC42F6D3F7F7CEFED8A40008F8A4000884
:108360002DE9F05F8246007800278B4615460AF11A
:108370000104B946302801D09DB113E014F8010B77
:108380000127782803D0582801D045B10AE00DB163
:10839000102D07D10027102514F8010B02E0082545
:1083A00000E00A250026B0460EE005FB080005FBAC
:1083B00006F1012701EB10461FFA80F8B6F5803F61
:1083C00000D3B94614F8010B294600F069F80028DB
:1083D000EBDABBF1000F05D00FB1641E00E054468C
:1083E000CBF80040B9F1000F06D000F0BDF8022133
:1083F0000160C81EBDE8F09F48EA0640FAE72DE993
:10840000F04D00231A461B1A8A4103DB0020014667
:10841000BDE8F08DC1F30A52C1F3130141F4801598
:108420004FF0000BD10702D100186D41521E0026FB
:10843000044640F2FF11304601EB620A374680469F
:10844000024600204FF48011FFF77FFD801979412B
:10845000331847EB0102B4EB030C75EB020C04D3A9
:10846000E41A65EB020506460F46241908F10100DF
:108470006D4180463428E3DDB11947EB0700091B45
:10848000A84103D24FF0FF32134601E00022134609
:108490001BEB060047EB0A51BDE8F04DFFF744BE69
:1084A0003A2800D2303820F02002412A01D3A2F12C
:1084B0003700884201D34FF0FF30704770B501EBB1
:1084C000020410F8015B15F0070301D110F8013B1D
:1084D0002A1106D110F8012B03E010F8016B01F806
:1084E000016B5B1EF9D12B0705D40023521E0FD45C
:1084F00001F8013BFAE710F8013B02F10202A1EB9F
:10850000030303E013F8015B01F8015B521EF9D588
:10851000A142D6D3002070BD490050EAC12018BF47
:1085200004204A0D18BF40F0010040F2FF72B2EB88
:10853000515F08BF40F00200012808BF05207047C6
:108540004100080218BF04200A0E18BF40F00100C5
:108550004FF07F4232EA010108BF40F002000128DB
:1085600008BF0520704700000048704774040020D1
:108570002DE9F0414F1E00EBC7010446D1E900018F
:1085800015461E4637F006020DD02A463346FFF741
:10859000E2FB7F1E04EBC703D3E90023FFF735FBA3
:1085A00037F00602F1D1022F25D0042F13D0062F69
:1085B00018BFBDE8F0812A463346FFF7CCFBD4E96B
:1085C0000A23FFF722FB2A463346FFF7C4FBD4E910
:1085D0000823FFF71AFB2A463346FFF7BCFBD4E912
:1085E0000623FFF712FB2A463346FFF7B4FBD4E914
:1085F0000423FFF70AFB2A463346FFF7ACFBD4E916
:108600000223FFF702FB2A463346FFF7A4FBD4E917
:108610000023BDE8F041FFF7F8BA0000024A00204D
:108620001107FFF74FBE000001FDFFFF6FF05E0175
:108630000807FFF720BD00002DE9F04D0346144662
:108640004FF07F400E46B0EB440F04D80016086090
:108650001846BDE8F08D4FF0004040EA0421C4F315
:10866000C7507838431100F01F00DFF814C1C0F183
:108670002002FC445CF823500CEB83038540D3F8C4
:1086800004C02CFA02F72F439D680CFA00FC25FA6F
:1086900002F8DB6805FA00F023FA02F240EA02056C
:1086A0004CEA080CA7FB0123ACFB01C0A5FB015160
:1086B00001EB0C05A94294BF4FF0000C4FF0010CE8
:1086C00081186144BCF1000F02D0814202D903E05D
:1086D000814201D2012000E00020184400F1200274
:1086E0004FEA92188006CA0C40EA42304F03C6F89F
:1086F0000080FFF7A0FB82463846FFF7A5FB6FF02E
:108700001201FFF7B8FC07462846FFF79DFB6FF004
:108710002501FFF7B0FC834639465046FFF7A7F91D
:108720005946FFF7A4F900F500656FF30B055146B4
:108730002846FFF7EEF93946FFF7EBF95946FFF700
:10874000EBF91049FFF7EBF907460F492846FFF709
:10875000E6F93946FFF78BF907460C492846FFF73B
:10876000DEF93946FFF783F914F0004F08BFBDE882
:10877000F08DC8F1805180F000403160BDE8F08D8F
:1087800002190000DB0FC92F22AAFD290000C92F02
:1087900002E008C8121F08C1002AFAD170477047CA
:1087A000002001E001C1121F002AFBD17047000028
:1087B0000149086070470000740400202DE9F0476B
:1087C0004FF0684202EB400305460C46B3F1654F9B
:1087D0003CBF02EB4102B2F1654F3FD34FF07F4205
:1087E000B2EB400F28BFB2EB410F03D2BDE8F04718
:1087F000FFF73DB940EA01035B0008BF44F0FF41C9
:108800000AD0B2EB400F08BFB2EB410F06D125F002
:10881000804024F0804105460C461FE0B2EB400F3B
:1088200012BF5FEA410245F0FF4004F0004115D05D
:108830004FEA410292EA400310D4002AACBF4FF045
:108840009F464FF03E563146FFF769F905463146DF
:108850002046FFF764F9044628462146C0F3C75274
:10886000C1F3C753D21A1B2A06DD10F0004F14BF04
:1088700054485548BDE8F08712F11A0F17DA11F085
:10888000004F06D010F0004F14BF50485048BDE8CC
:10889000F08721462846FFF778F90446FFF750FE97
:1088A000042808BFFFF7C2FE2046BDE8F08742005B
:1088B000B2EB410F25D910F0004F19BF454F464E7E
:1088C000464F474E224685F0004415460A4680F042
:1088D000004110460A1A5200B2F1807F3ED2484051
:1088E0004049DFF804A110F0004F18D04FF03F4886
:1088F0003846FFF70EF9074651463046FFF709F9AB
:1089000017E011F0004F04BF00263746E2D010F008
:10891000004F19BF354F364E364F374EDAE74FF01E
:108920007C583846FFF7A3F8074651463046FFF714
:108930009EF8064641462846FFF7F1F82146FFF724
:1089400096F8824621464046FFF7E9F82946FFF7A8
:10895000E3F85146FFF719F9044604E0214628469A
:10896000FFF713F904460146FFF7D9F8804623497B
:10897000FFF7D5F82249FFF77AF84146FFF7CFF81D
:108980002049FFF774F84146FFF7C9F81E49FFF781
:108990006EF84146FFF7C3F81C49FFF768F8054633
:1089A00041462046FFF7BBF82946FFF7B8F83146A5
:1089B000FFF75DF82146FFF75AF83946BDE8F04762
:1089C000FFF755B8DB0FC9BFDB0FC93FDB0F49C04D
:1089D000DB0F49400000C9BF22AAFDB90000C93F12
:1089E00022AAFD390060ED3EC30ACE37000049C01F
:1089F00022AA7DBA0000494022AA7D3A2DAD65BD6C
:108A00008FB8D53D0FB511BE61C84C3EA8AAAABE0D
:108A10002DE9F8430446024650486946B0EB420F40
:108A200009D94FF0E640B0EB420F8CBF4FF0FF305A
:108A30000020009034E04A4B22F0004083422BD9C2
:108A400048492046FFF76BF8FFF750FB0546FFF754
:108A500000FA00F00300009043492846FFF75FF852
:108A6000064642492846FFF75AF807464049284635
:108A7000FFF755F880463F492846FFF750F8214652
:108A8000FFF74AF84146FFF744F83946FFF741F847
:108A90003146FFF73EF802E01046FFF7CDFD0446F1
:108AA000009D002D18DA6000B0F17F4F3CBF4FF001
:108AB0007E50BDE8F88309D14FF00100FFF778FE42
:108AC000BDE8F84300210846FFF75FB82046BDE83F
:108AD000F8430121FFF7CFBA214615F0010F0846F0
:108AE0001DD0FFF71CF806462349FFF718F8234965
:108AF000FFF712F83146FFF712F82149FEF7B7FFEA
:108B00003146FFF70CF82146FFF709F82146FEF73A
:108B1000AEFF15F0020F18BFBDE8F8831AE0FEF7AC
:108B2000FEFF04461749FEF7FAFF1749FEF79FFFBD
:108B30002146FEF7F4FF1549FEF799FF2146FEF79F
:108B4000EEFF4FF07E51FEF792FF15F0020F08BFC7
:108B5000BDE8F88380F00040BDE8F883B61F927E40
:108B6000490E494683F9223F1A61342C0020A23372
:108B700000A0FD390000C93F336D4C39DA82083C52
:108B8000A0AA2ABEB93AB2BACA9F2A3DDDFFFFBEEB
:108B90002DE9F04D16460F460546020096B01C46DC
:108BA00021F0004123F0004014BF4FF0010C4FF0C2
:108BB000000C0CEB470CFE4B0CEB03084FEA630C6C
:108BC000C4452DD85FEA060818BF4FF0010808EB2E
:108BD00044089844F74B434522D8F74B50EA060C1B
:108BE00002D09F4205D14AB916B000201946BDE80F
:108BF000F08D002A08BF4FF0000C01D04FF0010C9F
:108C00000CEB470313F5001F0AD8002E14BF4FF0DA
:108C1000010C4FF0000C0CEB440313F5001F08D9B6
:108C200016B03246234628463946BDE8F04DFEF7D9
:108C3000ECBFDFF888B34FF0000A002FB8BF5845EB
:108C400023DADF4B9842A8BF4FF0020A1DDADA4B55
:108C500098421ADBDB4B03EB2053142B08DDC3F1E6
:108C6000340C26FA0CF303FA0CFCB4450DD108E0E1
:108C70005EB9C3F1140C20FA0CF303FA0CFC844522
:108C800003D103F00103C3F1020A51EA020321D127
:108C9000002C1FDA002F18BFBAF1020F02D0BAF170
:108CA000010F0BD00220FFF783FD16B00022BDE8B4
:108CB000F04D13461046C049FFF795BA0220FFF762
:108CC00077FD16B02A463B46BDE8F04D0020BA4974
:108CD000FFF789BA330076D1584525D107F1804096
:108CE00010F5801001BF002A0020B34916B008BF5C
:108CF000BDE8F08DB048814207DB002CA1BF1846CB
:108D0000214616B0BDE8F08D07E0201E05DA80F0A0
:108D1000004116B01846BDE8F08DAB497944D1E961
:108D2000000116B0BDE8F08DDFF88CC260452FD190
:108D3000002C28DA39B159451CD1002A04BF002083
:108D400002460CD01FE06AB10220FFF731FD40F26D
:108D5000013200204FF0E041FFF7B4FA0A463946ED
:108D600000F0DEBA954A394616B0002062F31E01C3
:108D7000BDE8F08D07DA16B03B46BDE8F04D0020A7
:108D80006146FFF730BA16B010463946BDE8F08D9F
:108D90008B4518DDB4F1804F0DD0A4F10053B3F131
:108DA000FF5310D13B1E0EDB16B01046BDE8F04D50
:108DB000194600F0A9BC3B4616B01046BDE8F04D80
:108DC0001946FEF7C8BF27F00043A2BBE1B15945E1
:108DD00038D1002F06DD002CA1BF0020594616B067
:108DE000BDE8F08D002F01DD002C1FDB002F16DA0F
:108DF000002C14DBBAF1010F4FF000000CBF7349D7
:108E00006E4916B0BDE8F08DBAF1020F18BF002F01
:108E10000CD0BAF1010F09D1002F07DA0CE0002FB6
:108E2000B8BF002C0EDABAF1010F05D0002016B041
:108E30000146BDE8F08D05E016B000204FF000417E
:108E4000BDE8F08D4FF0010C0CEBE7720F9252EA87
:108E50000A020BD05E4A90427DDD5E4B5E4A98422C
:108E600016DD91420EDC002C1CDB2CE00120FFF70C
:108E70009FFC16B00022BDE8F04D13461046114687
:108E8000FFF7B1B94C48884202DC002C0ADC1AE03A
:108E90008A4202DD002C05DB15E0474B99421EDDBE
:108EA000002C10DD0220FFF783FC40F2013200208D
:108EB0004FF0E041FFF706FA404A16B061F31E0298
:108EC0001146BDE8F08D0220FFF772FCFFF7A6FB0C
:108ED000394A16B061F31E021146BDE8F08D00223A
:108EE00028463946FEF731FF05460F466FF001026E
:108EF000FFF7E8F94FF05532384BFEF729FF2A46C5
:108F00003B46FEF728FF0022354BFEF721FF8B463C
:108F100080462A463B4610461946FEF71CFF42464D
:108F20005B46FEF718FF80460B914FF0C0422D4B79
:108F300028463946FEF70FFF834605912A4A294BFA
:108F400040460B99FEF707FF88460290274A284BB8
:108F50002846394600E01BE0FEF7FDFE4346029A34
:108F6000FEF7F3FE054602460B460B91584605995F
:108F7000FEF74BFE002788465A463846059BFEF70B
:108F8000E4FE2A460B9BFEF7E3FE024600F073B9AF
:108F90000020B1F5801F07DA352228461946FFF771
:108FA00091F905466FF0340000EB215022E00000FB
:108FB000FFFF1F00FFFF0F000000F03F0000F07FE9
:108FC0000000404301FCFFFF501200000000F0FFD2
:108FD0000000E0410000F043FFFFEF3F5555D53F53
:108FE0000000E03F4715F73FFE822B6544DF5DF848
:108FF0000BAE543EA0F2FF300190C1F3130040F0DD
:109000007F6141F040510291FE498842D8BF4FF044
:10901000000B0EDDFC498142C8BF4FF0010B08DC9C
:1090200001984FF0000B401C01900298A0F58010B1
:109030000290F6480299784400EBCB000991079022
:10904000D0E900232846FEF780FE0591009007989E
:10905000D0E9002328460999FEF7D7FD02460B46C2
:109060000020EB49FFF7BFF80B910B460246069034
:1090700005990098FEF76FFE0A90E648884600279B
:10908000784400680C9002994FF0005040EA61006B
:1090900000EB8B4000F5002102910798D0E90023F6
:1090A0000C98FEF752FE2A46099BFEF751FE3A46FF
:1090B0004346FEF750FE0791054638464146029B5F
:1090C0000C9AFEF748FE059B009AFEF741FE2A46E1
:1090D000079BFEF73AFE0B9B069AFEF73CFE0A9AA8
:1090E00006910890434610461946FEF734FE0546A1
:1090F0000246C9480B46079106217844FFF738FA23
:109100000290079B2A46059110461946FEF723FE5A
:10911000059B029AFEF71FFE059105464346384619
:1091200019460A9AFEF771FD069B089AFEF713FE90
:109130002A46059BFEF769FD3A4643460591129083
:1091400010461946FEF707FE0022B44B0791009027
:10915000FEF75BFD059B129AFEF757FD0D463A465A
:10916000AE4B3846FEF7F1FD079B009AFEF7EDFD8A
:10917000059B129AFEF7ECFD3A46079112902B469A
:1091800010464146FEF7E7FD0591009043460A9AD6
:1091900007991298FEF7DFFD804607912B463A4665
:1091A00006990898FEF7D7FD4246079BFEF72DFD6E
:1091B00088460690059B009AFEF727FD00200F4683
:1091C0000546059B009AFEF7C0FD4346069AFEF74A
:1091D000BFFD80460D914FF06042914B28463946C5
:1091E000FEF7B9FD059100908E4A8D4B40460D99D2
:1091F000FEF7B1FD804604918B4A8C4B28463946D8
:10920000FEF7A9FD4246049BFEF7FFFC884A7A441C
:1092100002EBCB03D3E90023FEF7F7FC02900491A5
:109220000198FFF766F80791DDE904310546029AD7
:109230000098FEF7EAFC7F4A7A4402EBCB0BDBE9AD
:109240000023FEF7E2FC2A46079BFEF7DEFC002720
:1092500088462A463846079BFEF777FDDBE9002360
:10926000FEF773FD059B009AFEF76FFD049B029AC3
:10927000FEF76EFD024600200A900F98644DAAF199
:109280000103184301D16C4D0A9000200B46029057
:1092900030462146FEF75FFD82468B462346304628
:1092A0001946029AFEF751FD3A464346FEF753FD32
:1092B00052465B46FEF7A9FC06468A463A464346B6
:1092C00021460298FEF747FD04460F4632465346B4
:1092D000FEF79BFC594A8B46914226DBABEB02031F
:1092E00053EA000210D122463B46FEF72EFD80468F
:1092F0000391534A534B30465146FEF786FC424693
:10930000039BFFF707F82CD20220FFF751FA40F237
:10931000013200204FF0E041FEF7D4FF0A46294613
:1093200016B062F31E01BDE8F08D474B2BF00042F2
:109330009A4216D3454A0BEB020353EA000208D1C6
:1093400022463B46FEF701FD32465346FEF7E2FF5A
:1093500007D80220FFF72CFAFFF760F90A462946E2
:10936000DEE72BF000403A493A4A01EB20514FF03A
:109370000008904223DD481C4FF4801121FA00F0D0
:109380005844C0F30A51344AA1F2FF317A44334BB6
:109390001268CB4020EA0303C0F3130040F4801CA2
:1093A000C1F114002CFA00F8BBF1000FB8BFC8F1EE
:1093B000000820463946FEF7C8FC04460F46224600
:1093C0003B4630465146FEF720FC4FF0000B5A4614
:1093D000234B58460791FEF7BEFC05910090214AA9
:1093E000214B58460799FEF7B6FCCDE9020122460B
:1093F0003B4658460799FEF7A8FC32465346FEF70F
:10940000A7FC33E08E9803007AB60B00260E00000E
:109410000000F03FEC0E0000920D0000000008403C
:1094200009C7EE3FFD033ADCF5015B14E02F3EBEB9
:109430006E0C0000340C00000000F0BF00009040F3
:10944000FE822B654715973C00CC904000346F3F5F
:1094500001FCFFFF0000E03FE00B0000FFFF0F00FA
:10946000432EE63F396CA80C615C20BE3F4A404B5E
:10947000FEF771FCDDE90223FEF7C7FB07468A46CB
:10948000059B009AFEF7C1FB04460E46059B009A19
:10949000FEF75BFC3A465346FEF75AFC0746224667
:1094A00033460B9110461946FEF755FC834602469B
:1094B00030488A460B4605217844FFF759F85A464A
:1094C0005346FEF748FC22463346FEF741FC8246EF
:1094D0008B463A46204631460B9BFEF73CFC3A460B
:1094E0000B9BFEF792FB00910C9000224FF0804303
:1094F00050465946FEF729FC0746039152465B4603
:1095000020463146FEF727FC3A46039BFEF76BFEEA
:10951000009B0C9AFEF719FC22463346FEF715FC19
:109520000022154BFEF714FC0E46044601EB0851D1
:109530000815002810DC424620463146FEF7C2FEE0
:10954000FEF7EAFF042808BFFFF768F84246204606
:109550003146FEF7B7FE04460A980B4616B022467F
:109560002946BDE8F04DFEF7F6BB0000EF39FAFEE4
:10957000422EE63F040A00000000F03F2DE9F843C8
:109580000446544822466946B0EB420F09D94FF0D1
:10959000E640B0EB440F8CBF4FF0FF30002000904E
:1095A00034E04D4B22F0004083422BD94B4910460A
:1095B000FEF7B5FAFEF79AFD0646FEF74AFC00F004
:1095C0000300009046493046FEF7A9FA0546454992
:1095D0003046FEF7A4FA074643493046FEF79FFAA5
:1095E000804642493046FEF79AFA2146FEF794FA41
:1095F0004146FEF78EFA3946FEF78BFA2946FEF70A
:1096000088FA02E01046FFF717F80446009D002D87
:109610001DDA6000B0F17F4F09D22046FEF790FFBF
:10962000042808BFFFF702F82046BDE8F88308D1F8
:109630000120FFF7BDF8BDE8F84300210846FEF71A
:10964000A4BA2046BDE8F8430121FEF714BD214627
:1096500015F0010F08461FD0FEF761FA04462449B1
:10966000FEF75DFA2349FEF702FA2146FEF757FAA4
:109670002149FEF7FCF92146FEF751FA4FF07E51E1
:10968000FEF7F5F915F0020F08BFBDE8F88300BF3B
:1096900080F00040BDE8F883FEF741FA064617491E
:1096A000FEF73DFA1649FEF737FA3146FEF737FA6C
:1096B0001449FEF7DCF93146FEF731FA2146FEF790
:1096C0002EFA2146FEF7D3F915F0020FE0D1BDE8DE
:1096D000F8830000B61F927E490E494683F9223F67
:1096E0001A61342C0020A23300A0FD390000C93FCC
:1096F000B93AB2BACA9F2A3DDDFFFFBE336D4C397D
:10970000DA82083CA0AA2ABE2DE9F04106460F469F
:10971000FEF775FE0D46040018BF0120284320F017
:109720000040C0F17F6010F1E0400FD5002E14BF63
:1097300001200020384320F00040C0F17F6000F19C
:10974000E0400028A4BF0120FFF732F82046294658
:10975000BDE8F08170B50546FEF799FC044620F09F
:109760000040C0F1FF40C00F08D025F00040C0F11C
:10977000FF40C00F04BF0120FFF71AF8204670BD5C
:10978000BFA3000814A4000867010008EDA30008A7
:10979000D7A40008AF01000890A1000867A2000844
:1097A000D30100085CA30008D7A40008A1020008A8
:1097B00058A3000861A30008E10200087DA3000887
:1097C00031A4000855030008E1A1000804A4000822
:1097D0008B010008E9A3000844A400085D04000808
:1097E000E2A30008D6A300083D07000813A3000861
:1097F000D7A4000829080008EFA000080000000016
:109800000D0500200000000020000000ECA0000872
:10981000000000000E0500200000000064000000B1
:109820004DA20008000000000F050020010000000C
:10983000FA000000A6A000080200000012050020A7
:10984000B0040000A406000062A1000802000000AD
:109850001E05002000000000D00700006EA10008D7
:10986000020000002005002000000000D0070000DA
:10987000F8A00008020000002205002000000000FF
:10988000D00700003BA200080200000014050020E1
:1098900000000000D007000044A200080200000001
:1098A0001605002000000000D0070000A8A2000854
:1098B000000000001805002000000000010000006A
:1098C000B6A40008000000001905002000000000F8
:1098D000C8000000C5A40008000000001A05002010
:1098E00000000000C800000050A1000802000000B5
:1098F0001C050020E8030000D0070000A7A1000815
:10990000020000002405002032000000F2010000E7
:1099100098A1000802000000260500203200000087
:10992000F2010000C4A10008040000006805002046
:10993000B004000000C20100D4A10008040000002F
:1099400058050020B004000000C20100A3A30008D5
:1099500000000000100500200000000001000000D1
:1099600037A1000800000000020500200A000000E6
:10997000C800000016A10008000000000305002038
:109980000A0000003200000003A1000800000000EF
:10999000040500200A000000320000002BA300088C
:1099A0000100000040050020FFFFFFFF0100000054
:1099B00041A1000802000000420500200000000054
:1099C000D007000007A300080200000044050020A3
:1099D00000000000D0070000AAA400080200000058
:1099E0004605002000000000D0070000B2A30008D8
:1099F000000000004A05002000000000FF000000F9
:109A0000B5A2000801000000480500209CFFFFFFF0
:109A100064000000C7A20008010000004905002002
:109A20009CFFFFFF64000000E6A2000802000000A7
:109A30004C05002064000000B80B000089A4000859
:109A4000020000004E05002064000000B80B00007A
:109A5000CBA00008020000005005002064000000B8
:109A6000B80B0000F7A20008020000005205002019
:109A700064000000B80B00009AA400080200000077
:109A80005405002064000000B80B0000DCA00008B2
:109A9000020000005605002064000000B80B000022
:109AA00083A1000800000000DA040020000000008C
:109AB0000300000083A3000800000000DB04002076
:109AC00000000000FA000000E6A10008020000000B
:109AD000DC040020000000000001000092A3000848
:109AE00002000000DE04002064000000E803000023
:109AF00029A1000800000000E4040020000000008C
:109B0000010000001BA3000803000000D404002093
:109B1000B0B9FFFF5046000044A300080000000059
:109B2000A604002000000000C800000027A20008D2
:109B300000000000B004002000000000C800000089
:109B4000B7A0000800000000BA04002000000000D8
:109B5000C800000039A3000800000000A70400208E
:109B600000000000C80000001CA200080000000067
:109B7000B104002000000000C8000000ACA00008F4
:109B800000000000BB04002000000000C80000002E
:109B90004EA3000800000000A80400200000000000
:109BA000C800000031A2000800000000B20400203C
:109BB00000000000C8000000C1A000080000000074
:109BC000BC04002000000000C8000000C8A300087A
:109BD000020000005C05002000000000D00700002B
:109BE000EFA1000800000000600500200000000058
:109BF00001000000D8A20008020000006205002059
:109C00000A000000D00700007BA40008020000004A
:109C1000640500200A000000D0070000B6A100087B
:109C2000000000005F05002000000000640000004C
:109C30007AA1000802000000A0040020000000003B
:109C40002823000014A2000800000000A304002044
:109C500000000000C80000000CA200080000000086
:109C6000AD04002000000000C800000004A20008AD
:109C700000000000B704002000000000C800000041
:109C8000A1A2000800000000A204002000000000C3
:109C9000C80000009AA2000800000000AC040020E8
:109CA00000000000C800000093A2000800000000AF
:109CB000B604002000000000C80000006DA40008E9
:109CC00000000000A404002000000000C800000004
:109CD00067A4000800000000AE040020000000009F
:109CE000C800000061A4000800000000B8040020C3
:109CF00000000000C8000000FEA3000800000000F3
:109D0000A504002000000000C8000000F8A300081F
:109D100000000000AF04002000000000C8000000A8
:109D2000F2A3000800000000B904002000000000B9
:109D3000C80000008BA2000800000000A904002059
:109D400000000000C800000083A20008000000001E
:109D5000B304002000000000C80000007BA200083F
:109D600000000000BD04002000000000C80000004A
:109D70004145525431323334004143433B42415216
:109D80004F3B4D41473B43414D535441423B43417F
:109D90004D545249473B41524D3B47505320484F49
:109DA0004D453B47505320484F4C443B5041535343
:109DB000544852553B48454144465245453B42452F
:109DC000455045523B4C45444D41583B4C4C49470E
:109DD0004854533B4845414441444A3B00524F4C50
:109DE0004C3B50495443483B5941573B414C543BF1
:109DF000506F733B506F73523B4E6176523B4C45F4
:109E000056454C3B4D41473B56454C3B001048495D
:109E10004A4B4C4D44454647FF202122232425260A
:109E20002748494A4B4C4DFF1048498A8B8C8D84FA
:109E3000858687FF202122232425262748498A8BCF
:109E40008C8DFF00000C014008001000000C014048
:109E50001000100000080140001014000000000075
:109E6000000000000000F03F000000000000F83F8C
:109E700000000000000000000000004003B8E23FC6
:109E8000000000000000000006D0CF43EBFD4C3E78
:109E9000033333333333E33FFFAB6FDBB66DDB3F6D
:109EA0004D268F515555D53F01411DA96074D13FB5
:109EB00065DBC9934A86CD3FEF4E454A287ECA3FAF
:109EC0003E5555555555C53F93BDBE166CC166BF31
:109ED0002CDE25AF6A56113FF16BD2C541BDBBBE2A
:109EE000D0A4BE726937663E0040404040404040CA
:109EF000404041414141414040404040404040405D
:109F00004040404040404040400502020202020200
:109F1000020202020202020202202020202020204F
:109F20002020200202020202020290909090909063
:109F30001010101010101010101010101010101021
:109F40001010101002020202020288888888888895
:109F50000808080808080808080808080808080881
:109F6000080808080202020240000000E99E0008FA
:109F70000000000000000000000000006E83F9A255
:109F80002915444ED15727FCC0DD34F5999562DB85
:109F90004190433CAB6351FE4D5055363035300057
:109FA000565441494C34005934004144584C3334E0
:109FB000350048455836005936004F43544F5838FD
:109FC00000414343004641494C5341464500414905
:109FD00052504C414E45004D41470048454C495F69
:109FE00039305F444547004759524F5F534D4F4FFB
:109FF0005448494E47004C45445F52494E4700463D
:10A000004C59494E475F57494E4700424900545208
:10A01000490047494D42414C00494E464C4947484A
:10A02000545F4143435F43414C00435553544F4DAC
:10A030000048454C495F3132305F4343504D00503A
:10A04000504D005350454B5452554D004241524FD4
:10A05000005155414450004D4F544F525F53544F9F
:10A0600050004F43544F464C41545000534F4E41C3
:10A070005200475053005642415400534552564FE8
:10A080005F54494C54004845583658005155414496
:10A0900058004F43544F464C4154580054454C458A
:10A0A0004D45545259006D69647263006770735F67
:10A0B000706F73725F64006770735F706F735F645B
:10A0C000006770735F6E61765F640067696D6261DF
:10A0D0006C5F70697463685F6D69640067696D6265
:10A0E000616C5F726F6C6C5F6D696400796177643D
:10A0F00065616462616E64006D696E636F6D6D6150
:10A100006E6400766261746D696E63656C6C766F07
:10A110006C7461676500766261746D617863656C0B
:10A120006C766F6C74616765006D707536303530B4
:10A130005F7363616C6500766261747363616C6503
:10A14000007472695F7961775F6D6964646C650042
:10A150006661696C736166655F7468726F74746C54
:10A1600065006D696E7468726F74746C65006D6102
:10A17000787468726F74746C65006C6F6F7074695A
:10A180006D65006163635F68617264776172650029
:10A190006665617475726500736572766F5F70775E
:10A1A0006D5F72617465006D6F746F725F70776D53
:10A1B0005F72617465006E61765F736C65775F7264
:10A1C0006174650073657269616C5F626175647268
:10A1D000617465006770735F626175647261746554
:10A1E0000073617665006779726F5F6C7066006EF0
:10A1F00061765F636F6E74726F6C735F68656164C4
:10A20000696E6700645F706974636800695F706994
:10A2100074636800705F7069746368006770735F6F
:10A22000706F73725F69006770735F706F735F69DF
:10A23000006770735F6E61765F69006D696E636859
:10A2400065636B006D6178636865636B00616C7456
:10A250005F686F6C645F7468726F74746C655F6E56
:10A2600065757472616C006C697374206F72202D57
:10A2700076616C206F722076616C00645F6C65762D
:10A28000656C00695F6C6576656C00705F6C657607
:10A29000656C00645F726F6C6C00695F726F6C6CF0
:10A2A00000705F726F6C6C007265746172646564DB
:10A2B0005F61726D0067696D62616C5F7069746384
:10A2C000685F6761696E0067696D62616C5F726F7C
:10A2D0006C6C5F6761696E006E61765F7370656557
:10A2E000645F6D696E0067696D62616C5F7069744F
:10A2F00063685F6D696E0067696D62616C5F726F44
:10A300006C6C5F6D696E007472695F7961775F6D07
:10A31000696E0076657273696F6E006D61675F6468
:10A3200065636C696E6174696F6E007961775F64F3
:10A330006972656374696F6E006770735F706F73C5
:10A34000725F70006770735F706F735F700067702B
:10A35000735F6E61765F70006D61700068656C7030
:10A36000006D617070696E67206F66207263206394
:10A3700068616E6E656C206F72646572006D6978DD
:10A380006572006163635F6C70665F666163746FC2
:10A3900072006779726F5F636D70665F6661637488
:10A3A0006F72007370656B7472756D5F686972654A
:10A3B000730067696D62616C5F666C6167730064EE
:10A3C000656661756C7473006770735F77705F7238
:10A3D00061646975730073686F772073797374654E
:10A3E0006D207374617475730073657400657869AA
:10A3F0007400645F616C7400695F616C7400705F0D
:10A40000616C74007361766520616E6420726562B0
:10A410006F6F7400726573657420746F2064656675
:10A4200061756C747320616E64207265626F6F7405
:10A43000006D69786572206E616D65206F72206CA9
:10A44000697374006E616D653D76616C7565206F32
:10A450007220626C616E6B20666F72206C6973741F
:10A4600000645F79617700695F79617700705F7977
:10A470006177004D4D4138343578006E61765F73F9
:10A48000706565645F6D61780067696D62616C5FBE
:10A4900070697463685F6D61780067696D62616C93
:10A4A0005F726F6C6C5F6D6178007472695F796167
:10A4B000775F6D6178006661696C736166655F6482
:10A4C000656C6179006661696C736166655F6F6672
:10A4D000665F64656C617900F8A4000800000020E4
:10A4E00078040000BC84000814A60008780400204A
:10A4F00068180000A087000841130EA01B08510433
:10A500001A8C041A0B041A120413B79F1B08B20406
:10A510001AFF041AA7041A86141ABA081A62081A2B
:10A5200092041ACE0C1A31081ADB081AA0041A2A4F
:10A530000C411A3F081A76041A19041A43041A57D0
:10A54000041A7B041AE7241AF6041A720C1AC508B6
:10A550001A6C085A9C341AC1101A4C0C5AD7182974
:10A56000244113D7A41B08AA141A98041A730C4187
:10A5700002241A034B093D1204CBDC050201A00999
:10A5800012B00214030234018B803F0401CEE203B7
:10A59000124045080140018A1C1032029A04103210
:10A5A000049A081032082A0C104A041042408A1DEE
:10A5B000102A800B69104A0C609A081029602A0C36
:10A5C000103B2C01301129211A1B05691019612A31
:10A5D0000C104A083039602A1E454910396099101C
:10A5E0002940AA081019611A0C1013199E1B080D96
:10A5F000041A34041A28040138B93984A24A0438E8
:10A600000C01020304060708090204062329106945
:04A6100014410000F1
:04000005080000ED02
:00000001FF
